:020000040000FA
:04000000EEEF11F01E
:080008000B6E7F0B0BBC80089E
:10001000F76A200FF66E0800F5500BBE00081200BC
:10002000000306090C101316191C1F2225282B2E5D
:10003000313336393C3F414447494C4E5153555872
:100040005A5C5E60626466686A6B6D6F707173742F
:10005000757678797A7A7B7C7D7D7E7E7E7F7F7FE8
:100060007F001C6A1D6A01D0116E1250115ED8A06B
:1000700012061D501C5ED8A01D06D89011361236EF
:100080001C361D36031C0F6E041C106E0F2AD8B4CC
:10009000102A200E176E186A196A1A6A1B6A166AE5
:1000A0000F0EEA6E02C0E9FF071C87EC01F000D0DA
:1000B00000D0000011501826D8B0192A1250192665
:1000C0001C501A26D8B01B2A1D501B2619509CDF25
:1000D000800F0C6E1B5098DF800F0C260C301626FC
:1000E00002C0E9FFEF500710D8A00718EF6E170401
:1000F000D8B4200E176ED8B40F2AD8B4103ED7D774
:100100001200066A800E226E86EF00F0116A126AF3
:10011000136A146A089A12EC01F0D30FD8B4088A53
:100120002D0FC60FF8E20A0FF6E30F6E0E6A0D6A86
:100130000C6A0A0E0B6E65EC01F00F500B24116E69
:100140000C50126E000ED8B0010E12260D50136E18
:10015000000ED8B0010E13260E50146E000ED8B04B
:10016000010E1426060606E012EC01F0C60F02E2AC
:100170000A0FDBE208AA0BD0111E121E131E141E5A
:10018000112AD8B4122AD8B4132AD8B4142A115078
:100190001200066A116E126A00960650D8B40086E4
:1001A000050E056E270E106E100E0CD8030E106E85
:1001B000E80E08D8106A640E05D8106A0A0E02D834
:1001C000115008D00F6E12500C6E11500B6E4EEC89
:1001D00001F00B500B6E054E0096065003E0055CD7
:1001E000D8B008D00B50D8A4009600B603D0300F7A
:1001F00008EF01F01200A66AA68E0900F55002E091
:1002000002D8FBD712009EA8FED7AD6ED880120090
:1002100001B403EF01F001A205D001B003D001B297
:10022000EE6E120022BEEE501200AA6AA96EA66AF5
:10023000A680A850A94AAA2A1200AA6AA86EA66A8D
:10024000A684550EA76EAA0EA76EA682A6B2FED7EA
:10025000A694A94AAA2A1200106A0F6EFF0E0F2652
:10026000102200D0D8A01200030E0C6EE40E02D8AB
:10027000F5D70C6AF60F0B6E0C1ED8A006D0FE0E3A
:1002800000000B26D8B0FCD70B2600000C3EF7D799
:1002900000000BB000D00BB000D01200126A116A3F
:1002A000100EF36E0C34113612360F50115C1050D4
:1002B000125805E30F50115E1050125AD8800B36B9
:1002C0000C36F32EEFD70B501200200E156E1E6A5F
:1002D0001F6A206A216AD8900BA00ED011501E26EA
:1002E0001250D8B0123C1F261350D8B0133C202611
:1002F0001450D8B0143C2126213220321F321E3235
:100300000E320D320C320B32152EE5D71200E98871
:10031000E92AEC161200610EE75C05E67B0EE75C4D
:1003200002E7DF0EE716E650EE6EF5E11200A66A70
:10033000A68EEE500900F55C02E1F566FAD71200D0
:100340003D3D3D3D3D3D3D3D3D3D3D3D3D3D3D3DDD
:100350003D3D3D3D3D3D3D3D3D3D3D3D3D3D3D3DCD
:100360003D0055414920666F72204C41422D583264
:10037000207631206275696C642032360000434F6C
:100380005220676F657320696E61637469766500DA
:10039000434F5220676F657320616374697665000F
:1003A00050545420676F657320696E616374697679
:1003B000650050545420676F6573206163746976DB
:1003C0006500537461727420636F6D6D616E64209B
:1003D0006465636F64696E672E2E2E00696E6275A8
:1003E000663D000053657269616C20696E707574BA
:1003F00020627566666572206C656E677468203D64
:100400002000537061636520636861726163746585
:100410007220666F756E6420617420002D2D2D2D65
:100420002D2D2D2D2D2D2D2D2D2D2D2D2D2D2D2DFC
:100430002D2D2D2D2D2D2D2D2D2D2D2D0000436FEE
:100440006D6D616E6420737472696E67203D203C2F
:100450000000636D64203D200000617267203D2034
:10046000000050545444454C41590000435700008B
:100470004C495354544F4E450000544F4E450000D4
:1004800054455354544F4E450000504C544F4E4524
:100490004F4E0000504C544F4E454F464600484585
:1004A0004C5000004C4F4144000053415645000061
:1004B0005354415455530000525853544F50000068
:1004C000545853544F500000525853544152540002
:1004D00054585354415254005258544F4E453100D1
:1004E0005258544F4E4532005258544F4E453300E7
:1004F0005258544F4E4534005258544F4E453500D3
:10050000525854494D453100525854494D453200D6
:10051000525854494D453300525854494D453400C2
:10052000525854494D4535005258574149543100AD
:100530005258574149543200525857414954330098
:100540005258574149543400525857414954350084
:100550005458544F4E4531005458544F4E45320074
:100560005458544F4E4533005458544F4E45340060
:100570005458544F4E453500545854494D45310058
:10058000545854494D453200545854494D45330050
:10059000545854494D453400545854494D4535003C
:1005A0005458574149543100545857414954320026
:1005B0005458574149543300545857414954340012
:1005C000545857414954350044454255474F4E0011
:1005D0004465627567206D6F6465204F4E00444529
:1005E0004255474F46004465627567206D6F6465EC
:1005F000204F4646000052584D5554453100486939
:1006000067682052585F4D757465000052584D550B
:10061000544530004C6F772052585F4D757465001B
:10062000524553455400536574205054542064651A
:100630006C617920746F2000536574207278207487
:10064000656C656D6574727920746F6E65203120FC
:100650006672657175656E637920746F20005365ED
:10066000742072782074656C656D6574727920747D
:100670006F6E652032206672657175656E637920D4
:10068000746F20005365742072782074656C656DFA
:100690006574727920746F6E65203320667265719F
:1006A00075656E637920746F2000536574207278CD
:1006B0002074656C656D6574727920746F6E652049
:1006C00034206672657175656E637920746F2000E1
:1006D0005365742072782074656C656D65747279E9
:1006E00020746F6E652035206672657175656E6366
:1006F0007920746F20005365742072782074656CC3
:10070000656D6574727920746F6E65203120647533
:1007100072726174696F6E20746F2000536574206B
:1007200072782074656C656D6574727920746F6E73
:1007300065203220647572726174696F6E20746F07
:1007400020005365742072782074656C656D657443
:10075000727920746F6E65203320647572726174D3
:10076000696F6E20746F2000536574207278207456
:10077000656C656D6574727920746F6E65203420C8
:10078000647572726174696F6E20746F20005365B6
:10079000742072782074656C656D6574727920744C
:1007A0006F6E65203520647572726174696F6E209A
:1007B000746F20005365742072782064656C6179D1
:1007C000206265747765656E20746F6E65203120D8
:1007D000616E64203220746F20005365742072783B
:1007E0002064656C6179206265747765656E20743C
:1007F0006F6E65203220616E64203320746F20009C
:100800005365742072782064656C61792062657428
:100810007765656E20746F6E65203320616E64208D
:100820003420746F20005365742072782064656CE6
:100830006179206265747765656E20746F6E6520DE
:100840003420616E64203520746F2000536574205D
:1008500072782064656C6179206265747765656E75
:1008600020746F6E65207820616E64207920746F2B
:10087000202D204E6F742063757272656E746C79D2
:1008800020757365642E000053657420747820749D
:10089000656C656D6574727920746F6E65203120AA
:1008A0006672657175656E637920746F200053659B
:1008B000742074782074656C656D65747279207429
:1008C0006F6E652032206672657175656E63792082
:1008D000746F20005365742074782074656C656DA6
:1008E0006574727920746F6E65203320667265714D
:1008F00075656E637920746F200053657420747879
:100900002074656C656D6574727920746F6E6520F6
:1009100034206672657175656E637920746F20008E
:100920005365742074782074656C656D6574727994
:1009300020746F6E652035206672657175656E6313
:100940007920746F20005365742074782074656C6E
:10095000656D6574727920746F6E652031206475E1
:1009600072726174696F6E20746F20005365742019
:1009700074782074656C656D6574727920746F6E1F
:1009800065203220647572726174696F6E20746FB5
:1009900020005365742074782074656C656D6574EF
:1009A000727920746F6E6520332064757272617481
:1009B000696F6E20746F2000536574207478207402
:1009C000656C656D6574727920746F6E6520342076
:1009D000647572726174696F6E20746F2000536564
:1009E000742074782074656C656D657472792074F8
:1009F0006F6E65203520647572726174696F6E2048
:100A0000746F20005365742074782064656C61797C
:100A1000206265747765656E20746F6E6520312085
:100A2000616E64203220746F2000536574207478E6
:100A30002064656C6179206265747765656E2074E9
:100A40006F6E65203220616E64203320746F200049
:100A50005365742074782064656C617920626574D4
:100A60007765656E20746F6E65203320616E64203B
:100A70003420746F20005365742074782064656C92
:100A80006179206265747765656E20746F6E65208C
:100A90003420616E64203520746F2000536574200B
:100AA00074782064656C6179206265747765656E21
:100AB00020746F6E65207820616E64207920746FD9
:100AC000202D204E6F742063757272656E746C7980
:100AD00020757365642E000053657420727820754C
:100AE0006E6B65792074656C656D657472792073C1
:100AF000746172742064656C61792074696D65201D
:100B0000746F200053657420727820756E6B657960
:100B10002074656C656D657472792073746F7020D4
:100B200064656C61792074696D6520746F200000C4
:100B30005365742074782074656C656D6574727982
:100B40002073746172742064656C61792074696DBE
:100B50006520746F20005365742074782074656C70
:100B6000656D657472792073746F702064656C6153
:100B7000792074696D6520746F2000005475726E61
:100B8000206F6E205445535420544F4E452E000084
:100B900053657420504C20746F6E6520656E636FD2
:100BA000646572206672657175656E637920746F15
:100BB0002000363700003639000037310000373466
:100BC0000000373700003739000038320000383570
:100BD000000038380000393100003934000039375E
:100BE00000003130300031303300313037003131E6
:100BF000300031313400313138003132330031329C
:100C00003700313331003133360031343100313483
:100C10003600313531003135360031353900313665
:100C2000320031363700313733003137390031384F
:100C3000330031383600313839003139320031393A
:100C4000360031393900323033003230360032313B
:100C5000300032313800323235003232390032332E
:100C60003300323431003235300032353400706CAC
:100C70005F66726571203D200000706C5F62697470
:100C80005F35203D2000706C5F6269745F34203DE9
:100C90002000706C5F6269745F33203D2000706CCF
:100CA0005F6269745F32203D2000706C5F6269741E
:100CB0005F31203D2000706C5F6269745F30203DC1
:100CC0002000736176655F7061726D733A20706C9D
:100CD0005F66726571203D20000057726974696E0D
:100CE0006720504C206672657175656E6379203D92
:100CF000200057726974696E6720434F5220646503
:100D00006C61792074696D65000057726974696E51
:100D100067205054542064656C61792074696D6556
:100D2000000057726974696E6720727820746F6E64
:100D3000652073746172742064656C617900577208
:100D40006974696E6720727820746F6E6520312037
:100D50006672657175656E63790057726974696E44
:100D60006720727820746F6E652031206C656E6725
:100D70007468000057726974696E67207278207712
:100D80006169742074696D6520310000577269745F
:100D9000696E6720727820746F6E652032206672EB
:100DA000657175656E63790057726974696E672045
:100DB000727820746F6E652032206C656E6774687F
:100DC000000057726974696E6720727820776169D4
:100DD000742074696D652032000057726974696E01
:100DE0006720727820746F6E65203320667265719B
:100DF00075656E63790057726974696E67207278E1
:100E000020746F6E652033206C656E677468000017
:100E100057726974696E67207278207761697420EF
:100E200074696D652033000057726974696E6720BC
:100E3000727820746F6E65203420667265717565F6
:100E40006E63790057726974696E672072782074D6
:100E50006F6E652034206C656E6774680000577291
:100E60006974696E6720727820776169742074698B
:100E70006D652034000057726974696E672072785E
:100E800020746F6E652035206672657175656E63BE
:100E9000790057726974696E6720727820746F6E7A
:100EA000652035206C656E67746800005772697440
:100EB000696E6720727820776169742074696D6546
:100EC0002035000057726974696E6720727820744B
:100ED0006F6E652073746F702064656C61790000BB
:100EE00057726974696E6720747820746F6E65201C
:100EF00073746172742064656C61790057726974EF
:100F0000696E6720747820746F6E65203120667278
:100F1000657175656E63790057726974696E6720D3
:100F2000747820746F6E652031206C656E6774680C
:100F3000000057726974696E672074782077616960
:100F4000742074696D652031000057726974696E90
:100F50006720747820746F6E652032206672657128
:100F600075656E63790057726974696E672074786D
:100F700020746F6E652032206C656E6774680000A7
:100F800057726974696E672074782077616974207C
:100F900074696D652032000057726974696E67204C
:100FA000747820746F6E6520332066726571756584
:100FB0006E63790057726974696E67207478207463
:100FC0006F6E652033206C656E6774680000577221
:100FD0006974696E67207478207761697420746918
:100FE0006D652033000057726974696E67207478EC
:100FF00020746F6E652034206672657175656E634E
:10100000790057726974696E6720747820746F6E06
:10101000652034206C656E677468000057726974CF
:10102000696E6720747820776169742074696D65D2
:101030002034000057726974696E672074782074D8
:101040006F6E652035206672657175656E63790017
:1010500057726974696E6720747820746F6E6520AA
:1010600035206C656E677468000057726974696E2C
:101070006720747820776169742074696D65203504
:10108000000057726974696E6720747820746F6EFF
:10109000652073746F702064656C61790000436F24
:1010A0006E66696775726174696F6E2073617665CB
:1010B0006420746F20666C617368206D656D6F725B
:1010C000792E000052656164696E6720636F6E66F9
:1010D000696775726174696F6E2066726F6D2066E4
:1010E0006C617368206D656D6F727900436F6E6619
:1010F000696775726174696F6E20726561642064DE
:101100006F6E652E0000706C5F66726571203D2009
:101110000000706C5F66726571203D200000617296
:1011200067203D20000053657420504C2066726596
:101130007175656E6379203D200053657420434FBF
:10114000522064656C61792074696D65203D2000D2
:10115000536574205054542064656C61792074691F
:101160006D65203D200053657420527820737461B2
:1011700072742064656C6179203D20005365742091
:10118000527820746F6E65203120667265717565C6
:101190006E6379203D2000005365742052782074DE
:1011A0006F6E65203120647572726174696F6E2094
:1011B0003D200000536574205278207761697420C7
:1011C00074696D652031203D20005365742052788C
:1011D00020746F6E652032206672657175656E636E
:1011E00079203D20000053657420527820746F6E82
:1011F00065203220647572726174696F6E203D20C3
:1012000000005365742052782077616974207469F6
:101210006D652032203D2000536574205278207483
:101220006F6E652033206672657175656E63792017
:101230003D20000053657420527820746F6E652045
:101240003320647572726174696F6E203D200000F6
:1012500053657420527820776169742074696D65D4
:101260002033203D200053657420527820746F6E27
:10127000652034206672657175656E6379203D2046
:10128000000053657420527820746F6E65203420FE
:10129000647572726174696F6E203D200000536541
:1012A0007420527820776169742074696D652034E8
:1012B000203D200053657420527820746F6E6520A5
:1012C00035206672657175656E6379203D2000007A
:1012D00053657420527820746F6E652035206475D4
:1012E00072726174696F6E203D2000005365742036
:1012F000527820776169742074696D652035203DCE
:1013000020005365742052782073746F70206465D8
:101310006C6179203D20000053657420547820735F
:10132000746172742064656C6179203D200053659E
:101330007420547820746F6E652031206672657158
:1013400075656E6379203D200000536574205478E4
:1013500020746F6E65203120647572726174696FDC
:101360006E203D2000005365742054782077616919
:10137000742074696D652031203D20005365742010
:10138000547820746F6E65203220667265717565C1
:101390006E6379203D2000005365742054782074DA
:1013A0006F6E65203220647572726174696F6E2091
:1013B0003D200000536574205478207761697420C3
:1013C00074696D652032203D200053657420547887
:1013D00020746F6E652033206672657175656E636B
:1013E00079203D20000053657420547820746F6E7E
:1013F00065203320647572726174696F6E203D20C0
:1014000000005365742054782077616974207469F2
:101410006D652033203D200053657420547820747E
:101420006F6E652034206672657175656E63792014
:101430003D20000053657420547820746F6E652041
:101440003420647572726174696F6E203D200000F3
:1014500053657420547820776169742074696D65D0
:101460002034203D200053657420547820746F6E22
:10147000652035206672657175656E6379203D2043
:10148000000053657420547820746F6E65203520F9
:10149000647572726174696F6E203D20000053653F
:1014A0007420547820776169742074696D652035E3
:1014B000203D20005365742054782073746F702091
:1014C00064656C6179203D200000436F6E6669673A
:1014D00075726174696F6E207265616420646F6EED
:1014E000652E000072785F73746172745F64656C5E
:1014F0006179203D200072785F746F6E655F315FA7
:1015000074696D65203D200072785F746F6E655F51
:10151000315F66726571203D200072785F77616986
:10152000745F315F74696D65203D200072785F746F
:101530006F6E655F325F74696D65203D2000727863
:101540005F746F6E655F325F66726571203D20006B
:1015500072785F776169745F325F74696D65203D91
:10156000200072785F746F6E655F335F74696D65BC
:10157000203D200072785F746F6E655F335F667226
:101580006571203D200072785F776169745F335F19
:1015900074696D65203D200072785F746F6E655FC1
:1015A000345F74696D65203D200072785F746F6EE2
:1015B000655F345F66726571203D200072785F77E9
:1015C0006169745F345F74696D65203D20007278D5
:1015D0005F746F6E655F355F74696D65203D2000D7
:1015E00072785F746F6E655F355F66726571203DFE
:1015F000200072785F776169745F355F74696D652B
:10160000203D200072785F73746F705F64656C6159
:1016100079203D20000074785F73746172745F6498
:10162000656C6179203D200074785F746F6E655F32
:10163000315F74696D65203D200074785F746F6E52
:10164000655F315F66726571203D200074785F7759
:101650006169745F315F74696D65203D2000747845
:101660005F746F6E655F325F74696D65203D200049
:1016700074785F746F6E655F325F66726571203D6E
:10168000200074785F776169745F325F74696D659B
:10169000203D200074785F746F6E655F335F7469FE
:1016A0006D65203D200074785F746F6E655F335FF9
:1016B00066726571203D200074785F776169745FA0
:1016C000335F74696D65203D200074785F746F6EC0
:1016D000655F345F74696D65203D200074785F74C8
:1016E0006F6E655F345F66726571203D20007478AF
:1016F0005F776169745F345F74696D65203D2000B8
:1017000074785F746F6E655F355F74696D65203DD9
:10171000200074785F746F6E655F355F6672657107
:10172000203D200074785F776169745F355F74696C
:101730006D65203D200074785F73746F705F646521
:101740006C6179203D200000417661696C61626CBA
:101750006520504C20656E636F64657220746F6EF7
:101760006573000036372E302020202020202039BD
:10177000342E38202020202020203133312E3820D4
:101780002020202020203137392E392020202020F1
:1017900020203231382E3120000036392E332020DF
:1017A000202020202039372E3420202020202020E7
:1017B0003133362E35202020202020203138332E82
:1017C00035202020202020203232352E37200000E6
:1017D00037312E392020202020203130302E30206B
:1017E0002020202020203134312E332020202020A2
:1017F00020203138362E3220202020202020323266
:10180000392E3120000037342E3420202020202093
:101810003130332E35202020202020203134362E28
:1018200032202020202020203138392E392020203D
:10183000202020203233332E3620000037372E3040
:101840002020202020203130372E32202020202040
:1018500020203135312E3420202020202020313905
:10186000322E38202020202020203234312E3820E3
:10187000000037392E372020202020203131302E13
:1018800039202020202020203135362E37202020DE
:10189000202020203139362E3620202020202020E4
:1018A0003235302E3320000038322E3520202020D3
:1018B00020203131342E38202020202020203135A6
:1018C000392E38202020202020203139392E352073
:1018D0002020202020203235342E312000003835C1
:1018E0002E342020202020203131382E3820202076
:1018F000202020203136322E32202020202020208F
:101900003230332E3520202020202020202020207F
:101910002020000038382E35202020202020313291
:10192000332E30202020202020203136372E392021
:101930002020202020203230362E3520202020204C
:101940002020202020202020000039312E3520208A
:10195000202020203132372E33202020202020202C
:101960003137332E38202020202020203231302ED5
:101970003720202020202020202020202020000090
:10198000456E746572206F6E6C7920746865206E88
:10199000756D62657220746F20746865206C656671
:1019A00074206F662074686520646563696D616C7E
:1019B00000004578616D706C653A2020746F20736B
:1019C0006574203132372E3320487A2C20656E74AE
:1019D000657220544F4E452031323700436F6D6D94
:1019E000616E642073756D6D61727900544F4E4560
:1019F000202020207878787820202053657420508B
:101A00004C20746F6E6520656E636F646572207420
:101A10006F207878787820487A0052585354415291
:101A20005420787878782020205365742074686575
:101A300020776169742074696D65206166746572D0
:101A4000207468652065787465726E616C20434F00
:101A5000522064726F7020696E70757420626566C2
:101A60006F7265207374617274696E672074686543
:101A700020756E6B65792074656C656D657472791F
:101A80002067656E65726174696F6E20787878780A
:101A9000206D732E00005258544F4E456E207878BA
:101AA000787820202053657420756E6B65792074DA
:101AB000656C656D6574727920746F6E65206E203B
:101AC000746F207878787820487A0000525854490A
:101AD0004D456E20787878782020205365742075E5
:101AE0006E6B65792074656C656D657472792074B0
:101AF0006F6E65206E206475726174696F6E2074FC
:101B00006F2078787878206D732E000052585741F6
:101B100049546E207878787820202053657420749A
:101B2000686520776169742074696D6520626574E9
:101B30007765656E2074656C656D65747279207467
:101B40006F6E65206E20616E6420746865206E651E
:101B5000787420746F6E6520746F207878787820A0
:101B60006D732E00525853544F5020207878787857
:101B70002020205365742074686520776169742083
:101B800074696D6520616674657220746865206C87
:101B90006173742074656C656D6574727920746FFF
:101BA0006E65206265666F72652064726F70706921
:101BB0006E6720434F522062792078787878206DC4
:101BC000732E00005458535441525420787878783A
:101BD0002020205365742074686520776169742023
:101BE00074696D652061667465722074686520652E
:101BF000787465726E616C20434F522064726F700E
:101C000020696E707574206265666F7265207374EA
:101C1000617274696E672074686520756E6B657992
:101C20002074656C656D657472792067656E657288
:101C30006174696F6E2078787878206D732E00005B
:101C40005458544F4E456E20787878782020205391
:101C5000657420756E6B65792074656C656D65744F
:101C6000727920746F6E65206E20746F207878789A
:101C70007820487A0000545854494D456E207878B1
:101C8000787820202053657420756E6B65792074F8
:101C9000656C656D6574727920746F6E65206E2059
:101CA0006475726174696F6E20746F2078787878CB
:101CB000206D732E00005458574149546E20787897
:101CC00078782020205365742074686520776169D6
:101CD000742074696D65206265747765656E207423
:101CE000656C656D6574727920746F6E65206E2009
:101CF000616E6420746865206E65787420746F6E00
:101D00006520746F2078787878206D732E00545891
:101D100053544F50202078787878202020536574D1
:101D20002074686520776169742074696D6520612D
:101D30006674657220746865206C617374207465C4
:101D40006C656D6574727920746F6E65206265666E
:101D50006F72652064726F7070696E6720434F52B6
:101D60002062792078787878206D732E00005054A6
:101D70005444454C41592078787878202053657434
:101D800020746865205054542064656C6179207417
:101D9000696D6520616674657220504C20656E63C4
:101DA0006F6465722073746F70732E0053544154C6
:101DB0005553202020202020202020446973706C5F
:101DC0006179207468652063757272656E74205540
:101DD000414920636F6E66696775726174696F6EE1
:101DE000000048454C50202020202020202020208A
:101DF00020446973706C6179207468697320686528
:101E00006C7020696E666F726D6174696F6E000030
:101E10004C495354544F4E4520202020202020442C
:101E20006973706C6179206C697374206F662073BC
:101E30007570706F7274656420504C20746F6E659D
:101E4000206672657175656E636965730000496E21
:101E50007465726E616C2074657374696E6720615D
:101E60006E6420646562756767696E6720636F6D75
:101E70006D616E647300504C544F4E454F4E2020A0
:101E800020202020205475726E206F6E20504C2030
:101E9000746F6E652067656E657261746F720000A5
:101EA000504C544F4E454F46462020202020205471
:101EB00075726E206F464620504C20746F6E652000
:101EC00067656E657261746F720054455354544F68
:101ED0004E452020202020202047656E65726174C9
:101EE000652031204B687A20746F6E6520666F72B2
:101EF0002035207365636F6E64730000444542555E
:101F0000474F4E20202020202020205475726E2024
:101F10006F6E20646562756767696E67206D6573B3
:101F200073616765730044454255474F464620201C
:101F300020202020205475726E206F666620646514
:101F400062756767696E67206D6573736167657336
:101F5000000052584D55544531202020202020208B
:101F6000204D75746520527820617564696F00009A
:101F700052584D55544530202020202020202050FC
:101F800061737320527820617564696F0000537427
:101F90006174757300002020504C20667265717565
:101FA000656E6379203D20002020434F52206465F8
:101FB0006C61792074696D65203D200020205054AB
:101FC000542064656C61792074696D65203D200042
:101FD00052782054656C656D657472792047656E22
:101FE00065726174696F6E0020205278207374618D
:101FF00072742064656C6179203D20002020527845
:1020000020746F6E652031206672657175656E6330
:1020100079203D2000002020527820746F6E6520CA
:102020003120647572726174696F6E203D2000000A
:102030002020527820776169742074696D652031A1
:102040002020202020203D200000202052782074D5
:102050006F6E652032206672657175656E637920DA
:102060003D2000002020527820746F6E65203220C1
:10207000647572726174696F6E203D2000002020CB
:10208000527820776169742074696D652032202050
:10209000202020203D2000002020527820746F6EE8
:1020A000652033206672657175656E6379203D2009
:1020B00000002020527820746F6E652033206475F4
:1020C00072726174696F6E203D200000202052788A
:1020D00020776169742074696D6520332020202089
:1020E00020203D2000002020527820746F6E652053
:1020F00034206672657175656E6379203D2000003D
:102100002020527820746F6E6520342064757272BE
:102110006174696F6E203D20000020205278207786
:102120006169742074696D6520342020202020208E
:102130003D2000002020527820746F6E65203520ED
:102140006672657175656E6379203D200000202000
:10215000527820746F6E65203520647572726174D8
:10216000696F6E203D200000202052782077616941
:10217000742074696D6520352020202020203D20AA
:102180000000202052782073746F702064656C61A9
:1021900079202020202020203D2000005478205449
:1021A000656C656D657472792047656E65726174E2
:1021B000696F6E00202054782073746172742064FB
:1021C000656C61792020202020203D200000202007
:1021D000547820746F6E6520312066726571756564
:1021E0006E6379203D2000002020547820746F6EAB
:1021F00065203120647572726174696F6E203D20B4
:1022000000002020547820776169742074696D651E
:1022100020312020202020203D2000002020547844
:1022200020746F6E652032206672657175656E630D
:1022300079203D2000002020547820746F6E6520A6
:102240003220647572726174696F6E203D200000E7
:102250002020547820776169742074696D6520327C
:102260002020202020203D200000202054782074B1
:102270006F6E652033206672657175656E637920B7
:102280003D2000002020547820746F6E652033209C
:10229000647572726174696F6E203D2000002020A9
:1022A000547820776169742074696D65203320202B
:1022B000202020203D2000002020547820746F6EC4
:1022C000652034206672657175656E6379203D20E6
:1022D00000002020547820746F6E652034206475CF
:1022E00072726174696F6E203D2000002020547866
:1022F00020776169742074696D6520342020202066
:1023000020203D2000002020547820746F6E65202E
:1023100035206672657175656E6379203D20000019
:102320002020547820746F6E652035206475727299
:102330006174696F6E203D20000020205478207762
:102340006169742074696D6520352020202020206B
:102350003D200000202054782073746F7020646545
:102360006C6179202020202020203D200000436F38
:102370006E66696775726174696F6E2072656164FB
:1023800020646F6E652E0000456E746572204C49A6
:102390005354544F4E4520746F206C6973742073EE
:1023A0007570706F7274656420504C20746F6E6528
:1023B000732E0000526573657420616C6C2070612F
:1023C00072616D657465727320746F2064656661F7
:1023D000756C742076616C7565732E00F86A006AFE
:1023E000400EAF6E200EAC6E900EAB6E0F0EAF6E49
:1023F000900EAB6E200EAC6E070EB46E0F0EC16E5B
:10240000F19E93948194939081909392819294966B
:102410008296949882980101B96BBA6B00013EECE8
:1024200019F028EC19F0246A01016D916D936A6B23
:10243000010E696F736B726B716B706B6D85B89702
:102440006D896D87010E106EF40E2DEC01F00D0EEE
:1024500003EC01F00A0E03EC01F0030EF76E400EE0
:10246000F66EFBEC00F00D0E03EC01F00A0E03EC2F
:1024700001F0030EF76E620EF66EFBEC00F00D0E2F
:1024800003EC01F00A0E03EC01F0820E026E040E62
:10249000076E046A0A0E036E126A640E116E31EC46
:1024A00000F0820E026E020E076E046A0A0E036EC0
:1024B000126A640E116E31EC00F000013DEC2EF05A
:1024C00050EC23F0320E2CEC01F0010E81B6E86ADC
:1024D000236E010E01016DB1E86A23140001D8B426
:1024E00074EF12F092EF13F0010E81B6E86A236EDA
:1024F000E86A01016DB1010E23140001D8B483EF25
:1025000012F03AEF13F0E86A81B6010E236E010E65
:1025100001016DB1E86A23140001D8B492EF12F002
:102520006AEF13F0E86A81B6010E236EE86A0101D2
:102530006DB1010E23140001D8B4A1EF12F0A6EF83
:1025400013F0ACEF12F081A8AAEF12F093928192EF
:10255000ACEF12F09392818281A8B3EF12F09392C4
:102560008182B5EF12F093928192D89601016DB5F8
:10257000D8860001D8B6BFEF12F094968286D8961E
:1025800001016DA5D8860001D8B6C9EF12F0949666
:102590008296010E82BAE86A236E010E01016DB3C4
:1025A000E86A23140001D8B4D8EF12F021EF14F038
:1025B000010E82BAE86A236EE86A01016DB3010E6A
:1025C00023140001D8B4E7EF12F0BAEF13F0E86A71
:1025D00082BA010E236E010E01016DB3E86A231465
:1025E0000001D8B4F6EF12F0F1EF13F0E86A82BA06
:1025F000010E236EE86A01016DB3010E2314000180
:10260000D8B405EF13F033EF14F00EEC13F02452AE
:10261000D8B40DEF13F01CEC13F057D7246A9EAA20
:1026200014EF13F0AECF24F012009EB819EF13F0A0
:10263000FCD724C0ADFF12000D0E245CD8B426EFE9
:1026400013F00A0E245CD8A42AEF13F060EC14F007
:1026500039EF13F0200E245CD8A038EF13F07F0E72
:10266000245CD8B038EF13F057EC14F039EF13F0C6
:10267000DCDF1200D8960101B8A7D8860001D8B6D1
:102680004EEF13F0030EF76E7E0EF66EFBEC00F0CD
:102690000D0E03EC01F00A0E03EC01F09498828811
:1026A00001016D91D8966DA9D8860001D8B65BEF6F
:1026B00013F058EC37F061EF13F09390818063EFE3
:1026C00013F0939081909390819069EF13F0939021
:1026D000818037D7D8960101B8A7D8860001D8B62F
:1026E0007EEF13F0030EF76E900EF66EFBEC00F02B
:1026F0000D0E03EC01F00A0E03EC01F094988298A1
:102700009390818086EF13F0939081908CEF13F07B
:10271000939081908EEF13F09390818001016D81F1
:1027200000010FD79498828801016D9100019DEFFF
:1027300013F0939081809FEF13F09390819093908A
:102740008190A5EF13F093908180FBD694988298A6
:1027500001016D810001B1EF13F093908190B3EF0F
:1027600013F09390818093908180B9EF13F0939050
:102770008190E7D6D8960101B8A7D8860001D8B6CF
:10278000CEEF13F0030EF76EA00EF66EFBEC00F02A
:102790000D0E03EC01F00A0E03EC01F001016D9344
:1027A000D8966DA7D8860001D8B6D9EF13F06BEC98
:1027B0003AF0949682866FC110F001016E512DECB3
:1027C00001F0939481940001E8EF13F093948184D5
:1027D000EEEF13F093948184F0EF13F093948194CF
:1027E00014D7D8960101B8A7D8860001D8B605EF4E
:1027F00014F0030EF76EB20EF66EFBEC00F00D0E49
:1028000003EC01F00A0E03EC01F0D89601016DA56E
:10281000D8860001D8B60FEF14F094968296939460
:10282000819415EF14F0939481841BEF14F093942A
:1028300081841DEF14F09394819401016D83000154
:10284000E4D601016D939394819400012AEF14F072
:102850009394818430EF14F09394818432EF14F0D8
:1028600093948194D2D601016D83D8966DA5D886B4
:102870000001D8B63EEF14F094968296D8960101E6
:102880006DB5D8860001D8B648EF14F094968286CC
:10289000939481844EEF14F09394819454EF14F048
:1028A0009394819456EF14F093948184AED600EE05
:1028B00025F0EE50FEE1ED5224C0EEFFEF6A12006B
:1028C0003EEC19F0D8960101B8A7D8860001D8B619
:1028D0007CEF14F00D0E03EC01F00A0E03EC01F096
:1028E000030EF76EC20EF66EFBEC00F00D0E03EC5D
:1028F00001F00A0E03EC01F0D8960101B8A7D886C2
:102900000001D8B697EF14F0030EF76EDC0EF66EEA
:10291000FBEC00F000EE25F0EE5003E003EC01F0DC
:10292000FBD70D0E03EC01F00A0E03EC01F025526B
:10293000D8A49CEF14F012000101B96B0001400E05
:102940000101B95D0001D8B0B5EF14F000EE25F03B
:102950000101B951EBCF09F000EE66F0B95109C0A1
:10296000EBFFB92B0001D8A4E9D728EC19F0BAEC99
:1029700014F0120000EE66F0E86AEE5202E0E83E63
:10298000FCD70101BA6F00EE66F0E86AEE5202E091
:10299000E83EFCD7096EB96B00010101B951095C31
:1029A0000001D8A0E9EF14F000EE66F00101B95182
:1029B000EB500A6E200E0A5C0001D8A4E4EF14F07C
:1029C000B9C1BAF1E9EF14F00101B92B0001D8A4A3
:1029D000E3D7D8960101B8A7D8860001D8B630EF62
:1029E00015F000EE66F0E86AEE5202E0E83EFCD731
:1029F0000101BB6F01EEBCF0020E016EBB51C9ECD0
:102A000000F0EF6A030EF76EE40EF66EFBEC00F0DA
:102A100001EEBCF0EE5003E003EC01F0FBD70D0E2D
:102A200003EC01F00A0E03EC01F001EEBCF0020E23
:102A3000016EBA51C9EC00F0EF6A040EF76E020E97
:102A4000F66EFBEC00F001EEBCF0EE5003E003ECA0
:102A500001F0FBD70D0E03EC01F00A0E03EC01F0C0
:102A600000010101B96B00010B0E0101B95D00010C
:102A7000D8B046EF15F0F36A00EEE9F00101B95164
:102A8000F3CFEBFFB92B0001D8A4EDD70101B96B4F
:102A90000001360E0101B95D0001D8B05BEF15F001
:102AA000F36A00EEFEF00101B951F3CFEBFFB92B51
:102AB0000001D8A4EDD70101BA05096EB96B000178
:102AC0000101B951095C0001D8A076EF15F000EEC4
:102AD00066F00101B951EBCF0AF000EEE9F0B9510F
:102AE0000AC0EBFFB92B0001D8A4E9D70101B96BEB
:102AF0000001360E0101B95D0001D8B094EF15F068
:102B00000101B951BA251C6E1D6A1D361C2800EE44
:102B100066F0EBCF09F000EEFEF0B95109C0EBFF13
:102B2000B92B0001D8A4E4D700EEE9F010EEE9F0EB
:102B30008BEC01F000EEFEF010EEFEF08BEC01F0FD
:102B4000D8960101B8A7D8860001D8B6F0EF15F0E5
:102B5000040EF76E1C0EF66EFBEC00F00D0E03EC8F
:102B600001F00A0E03EC01F0040EF76E3E0EF66E55
:102B7000FBEC00F000EE66F0EE5003E003EC01F039
:102B8000FBD73E0E03EC01F00D0E03EC01F00A0E34
:102B900003EC01F0040EF76E520EF66EFBEC00F043
:102BA00000EEE9F0EE5003E003EC01F0FBD70D0E70
:102BB00003EC01F00A0E03EC01F0040EF76E5A0E5E
:102BC000F66EFBEC00F000EEFEF0EE5003E003ECDE
:102BD00001F0FBD70D0E03EC01F00A0E03EC01F03F
:102BE000040EF76E620EF66E00EEE9F097EC01F05F
:102BF000D8A4FFEF15F054EC19F010EF19F0040E03
:102C0000F76E6C0EF66E00EEE9F097EC01F0D8A4CA
:102C10000EEF16F0DFEC44F010EF19F0040EF76E33
:102C2000700EF66E00EEE9F097EC01F0D8A41DEFFF
:102C300016F07AEC3DF010EF19F0040EF76E7A0EF4
:102C4000F66E00EEE9F097EC01F0D8A42CEF16F048
:102C500050EC23F010EF19F0040EF76E800EF66EB4
:102C600000EEE9F097EC01F0D8A43BEF16F01BEC76
:102C700023F010EF19F0040EF76E8A0EF66E00EED8
:102C8000E9F097EC01F0D8A44BEF16F001016D8547
:102C9000000110EF19F0040EF76E940EF66E00EEC0
:102CA000E9F097EC01F0D8A45BEF16F001016D9507
:102CB000000110EF19F0040EF76E9E0EF66E00EE96
:102CC000E9F097EC01F0D8A46AEF16F048EC44F074
:102CD00010EF19F0040EF76EA40EF66E00EEE9F098
:102CE00097EC01F0D8A479EF16F03DEC2EF010EF40
:102CF00019F0040EF76EAA0EF66E00EEE9F097ECEE
:102D000001F0D8A488EF16F0F7EC2AF010EF19F0D4
:102D1000040EF76EB00EF66E00EEE9F097EC01F0DF
:102D2000D8A497EF16F092EC3FF010EF19F0040ED4
:102D3000F76EB80EF66E00EEE9F097EC01F0D8A44D
:102D4000A6EF16F040EC22F010EF19F0040EF76E2B
:102D5000C00EF66E00EEE9F097EC01F0D8A4B5EFE6
:102D600016F0D2EC22F010EF19F0040EF76EC80E38
:102D7000F66E00EEE9F097EC01F0D8A4C4EF16F07F
:102D8000F7EC21F010EF19F0040EF76ED00EF66E8E
:102D900000EEE9F097EC01F0D8A4D3EF16F089EC3F
:102DA00022F010EF19F0040EF76ED80EF66E00EE5A
:102DB000E9F097EC01F0D8A4E2EF16F07DEC19F001
:102DC00010EF19F0040EF76EE00EF66E00EEE9F06B
:102DD00097EC01F0D8A4F1EF16F0C4EC19F010EF65
:102DE00019F0040EF76EE80EF66E00EEE9F097ECBF
:102DF00001F0D8A400EF17F00BEC1AF010EF19F067
:102E0000040EF76EF00EF66E00EEE9F097EC01F0AE
:102E1000D8A40FEF17F052EC1AF010EF19F0040ECF
:102E2000F76EF80EF66E00EEE9F097EC01F0D8A41C
:102E30001EEF17F099EC1AF010EF19F0050EF76E6F
:102E4000000EF66E00EEE9F097EC01F0D8A42DEF3D
:102E500017F0E0EC1AF010EF19F0050EF76E080EFF
:102E6000F66E00EEE9F097EC01F0D8A43CEF17F015
:102E700029EC1BF010EF19F0050EF76E100EF66E30
:102E800000EEE9F097EC01F0D8A44BEF17F072ECEC
:102E90001BF010EF19F0050EF76E180EF66E00EE2F
:102EA000E9F097EC01F0D8A45AEF17F0BBEC1BF057
:102EB00010EF19F0050EF76E200EF66E00EEE9F039
:102EC00097EC01F0D8A469EF17F004EC1CF010EFB8
:102ED00019F0050EF76E280EF66E00EEE9F097EC8D
:102EE00001F0D8A478EF17F04DEC1CF010EF19F0BA
:102EF000050EF76E300EF66E00EEE9F097EC01F07D
:102F0000D8A487EF17F096EC1CF010EF19F0050E1F
:102F1000F76E380EF66E00EEE9F097EC01F0D8A4EB
:102F200096EF17F0DFEC1CF010EF19F0050EF76EBE
:102F3000400EF66E00EEE9F097EC01F0D8A4A5EF94
:102F400017F028EC1DF010EF19F0050EF76E480E83
:102F5000F66E00EEE9F097EC01F0D8A4B4EF17F0AC
:102F600071EC1DF010EF19F0050EF76E500EF66EB5
:102F700000EEE9F097EC01F0D8A4C3EF17F0BAEC3B
:102F80001DF010EF19F0050EF76E580EF66E00EEFC
:102F9000E9F097EC01F0D8A4D2EF17F001EC1EF0A5
:102FA00010EF19F0050EF76E600EF66E00EEE9F008
:102FB00097EC01F0D8A4E1EF17F048EC1EF010EF09
:102FC00019F0050EF76E680EF66E00EEE9F097EC5C
:102FD00001F0D8A4F0EF17F08FEC1EF010EF19F00D
:102FE000050EF76E700EF66E00EEE9F097EC01F04C
:102FF000D8A4FFEF17F0D6EC1EF010EF19F0050E75
:10300000F76E780EF66E00EEE9F097EC01F0D8A4BA
:103010000EEF18F01DEC1FF010EF19F0050EF76E13
:10302000800EF66E00EEE9F097EC01F0D8A41DEFEB
:1030300018F066EC1FF010EF19F0050EF76E880E11
:10304000F66E00EEE9F097EC01F0D8A42CEF18F042
:10305000AFEC1FF010EF19F0050EF76E900EF66E44
:1030600000EEE9F097EC01F0D8A43BEF18F0F8EC93
:103070001FF010EF19F0050EF76E980EF66E00EEC9
:10308000E9F097EC01F0D8A44AEF18F041EC20F0F9
:1030900010EF19F0050EF76EA00EF66E00EEE9F0D7
:1030A00097EC01F0D8A459EF18F08AEC20F010EF5B
:1030B00019F0050EF76EA80EF66E00EEE9F097EC2B
:1030C00001F0D8A468EF18F0D3EC20F010EF19F05D
:1030D000050EF76EB00EF66E00EEE9F097EC01F01B
:1030E000D8A477EF18F01CEC21F010EF19F0050EC2
:1030F000F76EB80EF66E00EEE9F097EC01F0D8A48A
:1031000086EF18F065EC21F010EF19F0050EF76E60
:10311000C00EF66E00EEE9F097EC01F0D8A495EF42
:1031200018F0AEEC21F010EF19F0050EF76EC80E96
:10313000F66E00EEE9F097EC01F0D8A4B1EF18F0CC
:103140000101B887050EF76ED00EF66EFBEC00F0AD
:103150000D0E03EC01F00A0E03EC01F0000110EF7C
:1031600019F0050EF76EDE0EF66E00EEE9F097EC44
:1031700001F0D8A4CDEF18F00101B897050EF76E55
:10318000E60EF66EFBEC00F00D0E03EC01F00A0EFD
:1031900003EC01F0000110EF19F0050EF76EF60ECA
:1031A000F66E00EEE9F097EC01F0D8A4E8EF18F025
:1031B000050EF76EFE0EF66EFBEC00F00D0E03EC46
:1031C00001F00A0E03EC01F09498828810EF19F0D8
:1031D000060EF76E0C0EF66E00EEE9F097EC01F0BD
:1031E000D8A403EF19F0060EF76E140EF66EFBEC82
:1031F00000F00D0E03EC01F00A0E03EC01F09498C0
:10320000829810EF19F0060EF76E200EF66E00EEA3
:10321000E9F097EC01F0D8A410EF19F057EC44F066
:103220003EEC19F00D0E03EC01F00A0E03EC01F078
:10323000430E03EC01F06D0E03EC01F0640E03ECA1
:1032400001F03A0E03EC01F0200E03EC01F0120045
:103250000101B96B0001400E0101B95D0001D8B058
:103260003DEF19F0F36A00EE25F00101B951F3CFFB
:10327000EBFFB92B0001D8A4EDD712000101B96B07
:103280000001400E0101B95D0001D8B053EF19F003
:10329000F36A00EE66F00101B951F3CFEBFFB92BF1
:1032A0000001D8A4EDD71200060EF76E260EF66EBA
:1032B000FBEC00F000EEFEF0EE5003E003EC01F05A
:1032C000FBD7200E03EC01F06D0E03EC01F0730E42
:1032D00003EC01F02E0E03EC01F00D0E03EC01F0F7
:1032E0000A0E03EC01F000EEFEF081EC00F00101AB
:1032F0006E6F12C06FF100011200060EF76E380EED
:10330000F66EFBEC00F000EEFEF0EE5003E003EC96
:1033100001F0FBD7200E03EC01F0480E03EC01F0A6
:103320007A0E03EC01F00D0E03EC01F00A0E03EC33
:1033300001F000EEFEF081EC00F00101766F12C0AA
:1033400077F1775176110001D8A4ABEF19F00101A4
:10335000776B010E766F0001130E0101775D00019E
:10336000D8A0C2EF19F0D8A4BDEF19F0890E010161
:10337000765D0001D8A0C2EF19F0030E0101776F4E
:10338000E80E766F00011200060EF76E5E0EF66E06
:10339000FBEC00F000EEFEF0EE5003E003EC01F079
:1033A000FBD7200E03EC01F0480E03EC01F07A0E7F
:1033B00003EC01F00D0E03EC01F00A0E03EC01F03A
:1033C00000EEFEF081EC00F00101786F12C079F19F
:1033D000795178110001D8A4F2EF19F00101796B4D
:1033E000010E786F0001130E0101795D0001D8A074
:1033F00009EF1AF0D8A404EF1AF0890E0101785DE4
:103400000001D8A009EF1AF0030E0101796FE80E50
:10341000786F00011200060EF76E840EF66EFBEC5C
:1034200000F000EEFEF0EE5003E003EC01F0FBD7FD
:10343000200E03EC01F0480E03EC01F07A0E03ECD1
:1034400001F00D0E03EC01F00A0E03EC01F000EEAA
:10345000FEF081EC00F001017A6F12C07BF17B512C
:103460007A110001D8A439EF1AF001017B6B010E2B
:103470007A6F0001130E01017B5D0001D8A050EFAF
:103480001AF0D8A44BEF1AF0890E01017A5D000101
:10349000D8A050EF1AF0030E01017B6FE80E7A6F8F
:1034A00000011200060EF76EAA0EF66EFBEC00F09D
:1034B00000EEFEF0EE5003E003EC01F0FBD7200E2F
:1034C00003EC01F0480E03EC01F07A0E03EC01F07E
:1034D0000D0E03EC01F00A0E03EC01F000EEFEF01D
:1034E00081EC00F001017C6F12C07DF17D517C11F7
:1034F0000001D8A480EF1AF001017D6B010E7C6FF2
:103500000001130E01017D5D0001D8A097EF1AF0B4
:10351000D8A492EF1AF0890E01017C5D0001D8A0B9
:1035200097EF1AF0030E01017D6FE80E7C6F00012A
:103530001200060EF76ED00EF66EFBEC00F000EEF9
:10354000FEF0EE5003E003EC01F0FBD7200E03EC9D
:1035500001F0480E03EC01F07A0E03EC01F00D0EC1
:1035600003EC01F00A0E03EC01F000EEFEF081EC3A
:1035700000F001017E6F12C07FF17F517E110001CA
:10358000D8A4C7EF1AF001017F6B010E7E6F000116
:10359000130E01017F5D0001D8A0DEEF1AF0D8A460
:1035A000D9EF1AF0890E01017E5D0001D8A0DEEF8F
:1035B0001AF0030E01017F6FE80E7E6F000112000A
:1035C000060EF76EF60EF66EFBEC00F000EEFEF067
:1035D000EE5003E003EC01F0FBD7200E03EC01F00A
:1035E0006D0E03EC01F0730E03EC01F02E0E03ECF4
:1035F00001F00D0E03EC01F00A0E03EC01F000EEF9
:10360000FEF081EC00F00101806F12C081F1815168
:1036100080110001D8A411EF1BF00101816B010E94
:10362000806F0001130E0101815D0001D8A027EF1A
:103630001BF0D8A423EF1BF0890E0101805D00016F
:10364000D8A027EF1BF00101816B010E806F0001F4
:103650001200070EF76E1C0EF66EFBEC00F000EE8B
:10366000FEF0EE5003E003EC01F0FBD7200E03EC7C
:1036700001F06D0E03EC01F0730E03EC01F02E0E61
:1036800003EC01F00D0E03EC01F00A0E03EC01F067
:1036900000EEFEF081EC00F00101826F12C083F1B8
:1036A000835182110001D8A45AEF1BF00101836BF2
:1036B000010E826F0001130E0101835D0001D8A08D
:1036C00070EF1BF0D8A46CEF1BF0890E0101825D36
:1036D0000001D8A070EF1BF00101836B010E826F17
:1036E00000011200070EF76E420EF66EFBEC00F0C2
:1036F00000EEFEF0EE5003E003EC01F0FBD7200EED
:1037000003EC01F06D0E03EC01F0730E03EC01F01D
:103710002E0E03EC01F00D0E03EC01F00A0E03EC8B
:1037200001F000EEFEF081EC00F00101846F12C0A8
:1037300085F1855184110001D8A4A3EF1BF001018C
:10374000856B010E846F0001130E0101855D000180
:10375000D8A0B9EF1BF0D8A4B5EF1BF0890E01017A
:10376000845D0001D8A0B9EF1BF00101856B010E4B
:10377000846F00011200070EF76E680EF66EFBEC08
:1037800000F000EEFEF0EE5003E003EC01F0FBD79A
:10379000200E03EC01F06D0E03EC01F0730E03EC50
:1037A00001F02E0E03EC01F00D0E03EC01F00A0EF9
:1037B00003EC01F000EEFEF081EC00F00101866FF9
:1037C00012C087F1875186110001D8A4ECEF1BF0DD
:1037D0000101876B010E866F0001130E0101875DE9
:1037E0000001D8A002EF1CF0D8A4FEEF1BF0890E58
:1037F0000101865D0001D8A002EF1CF00101876B7A
:10380000010E866F00011200070EF76E8E0EF66E27
:10381000FBEC00F000EEFEF0EE5003E003EC01F0F4
:10382000FBD7200E03EC01F06D0E03EC01F0730EDC
:1038300003EC01F02E0E03EC01F00D0E03EC01F091
:103840000A0E03EC01F000EEFEF081EC00F0010145
:10385000886F12C089F1895188110001D8A435EF11
:103860001CF00101896B010E886F0001130E01012C
:10387000895D0001D8A04BEF1CF0D8A447EF1CF0E5
:10388000890E0101885D0001D8A04BEF1CF00101F9
:10389000896B010E886F00011200070EF76EB40EDF
:1038A000F66EFBEC00F000EEFEF0EE5003E003ECF1
:1038B00001F0FBD7200E03EC01F06D0E03EC01F0DC
:1038C000730E03EC01F02E0E03EC01F00D0E03EC71
:1038D00001F00A0E03EC01F000EEFEF081EC00F0C6
:1038E00001018A6F12C08BF18B518A110001D8A49B
:1038F0007EEF1CF001018B6B010E8A6F0001130E2D
:1039000001018B5D0001D8A094EF1CF0D8A490EFCA
:103910001CF0890E01018A5D0001D8A094EF1CF013
:1039200001018B6B010E8A6F00011200070EF76E0A
:10393000DA0EF66EFBEC00F000EEFEF0EE5003E067
:1039400003EC01F0FBD7200E03EC01F06D0E03EC4D
:1039500001F0730E03EC01F02E0E03EC01F00D0EDE
:1039600003EC01F00A0E03EC01F000EEFEF081EC36
:1039700000F001018C6F12C08DF18D518C1100018E
:10398000D8A4C7EF1CF001018D6B010E8C6F0001F4
:10399000130E01018D5D0001D8A0DDEF1CF0D8A44D
:1039A000D9EF1CF0890E01018C5D0001D8A0DDEF7C
:1039B0001CF001018D6B010E8C6F00011200080ECE
:1039C000F76E000EF66EFBEC00F000EEFEF0EE502F
:1039D00003E003EC01F0FBD7200E03EC01F06D0EC9
:1039E00003EC01F0730E03EC01F02E0E03EC01F07A
:1039F0000D0E03EC01F00A0E03EC01F000EEFEF0F8
:103A000081EC00F001018E6F12C08FF18F518E1189
:103A10000001D8A410EF1DF001018F6B010E8E6F15
:103A20000001130E01018F5D0001D8A026EF1DF0EB
:103A3000D8A422EF1DF0890E01018E5D0001D8A0EF
:103A400026EF1DF001018F6B010E8E6F0001120039
:103A5000080EF76E260EF66EFBEC00F000EEFEF0A0
:103A6000EE5003E003EC01F0FBD7200E03EC01F075
:103A70006D0E03EC01F0730E03EC01F02E0E03EC5F
:103A800001F00D0E03EC01F00A0E03EC01F000EE64
:103A9000FEF081EC00F00101906F12C091F19151A4
:103AA00090110001D8A459EF1DF00101916B010E96
:103AB000906F0001130E0101915D0001D8A06FEF1E
:103AC0001DF0D8A46BEF1DF0890E0101905D00017F
:103AD000D8A06FEF1DF00101916B010E906F0001F6
:103AE0001200080EF76E4C0EF66EFBEC00F000EEC6
:103AF000FEF0EE5003E003EC01F0FBD7200E03ECE8
:103B000001F06D0E03EC01F0730E03EC01F02E0ECC
:103B100003EC01F00D0E03EC01F00A0E03EC01F0D2
:103B200000EEFEF081EC00F00101926F12C093F103
:103B3000935192110001D8A4A2EF1DF00101936BE3
:103B4000010E926F0001130E0101935D0001D8A0D8
:103B5000B8EF1DF0D8A4B4EF1DF0890E0101925DFD
:103B60000001D8A0B8EF1DF00101936B010E926F18
:103B700000011200080EF76E880EF66EFBEC00F0E6
:103B800000EEFEF0EE5003E003EC01F0FBD7200E58
:103B900003EC01F0480E03EC01F07A0E03EC01F0A7
:103BA0000D0E03EC01F00A0E03EC01F000EEFEF046
:103BB00081EC00F00101986F12C099F199519811B0
:103BC0000001D8A4E8EF1DF00101996B010E986F78
:103BD0000001130E0101995D0001D8A0FFEF1DF057
:103BE000D8A4FAEF1DF0890E0101985D0001D8A05C
:103BF000FFEF1DF0030E0101996FE80E986F0001B1
:103C00001200080EF76EAE0EF66EFBEC00F000EE42
:103C1000FEF0EE5003E003EC01F0FBD7200E03ECC6
:103C200001F0480E03EC01F07A0E03EC01F00D0EEA
:103C300003EC01F00A0E03EC01F000EEFEF081EC63
:103C400000F001019A6F12C09BF19B519A11000183
:103C5000D8A42FEF1EF001019B6B010E9A6F00019B
:103C6000130E01019B5D0001D8A046EF1EF0D8A401
:103C700041EF1EF0890E01019A5D0001D8A046EFC8
:103C80001EF0030E01019B6FE80E9A6F00011200F7
:103C9000080EF76ED40EF66EFBEC00F000EEFEF0B0
:103CA000EE5003E003EC01F0FBD7200E03EC01F033
:103CB000480E03EC01F07A0E03EC01F00D0E03EC5C
:103CC00001F00A0E03EC01F000EEFEF081EC00F0D2
:103CD00001019C6F12C09DF19D519C110001D8A45F
:103CE00076EF1EF001019D6B010E9C6F0001130E1B
:103CF00001019D5D0001D8A08DEF1EF0D8A488EFD2
:103D00001EF0890E01019C5D0001D8A08DEF1EF010
:103D1000030E01019D6FE80E9C6F00011200080E5A
:103D2000F76EFA0EF66EFBEC00F000EEFEF0EE50D1
:103D300003E003EC01F0FBD7200E03EC01F0480E8A
:103D400003EC01F07A0E03EC01F00D0E03EC01F030
:103D50000A0E03EC01F000EEFEF081EC00F0010130
:103D60009E6F12C09FF19F519E110001D8A4BDEF1C
:103D70001EF001019F6B010E9E6F0001130E0101E9
:103D80009F5D0001D8A0D4EF1EF0D8A4CFEF1EF0A5
:103D9000890E01019E5D0001D8A0D4EF1EF0030E34
:103DA00001019F6FE80E9E6F00011200090EF76E71
:103DB000200EF66EFBEC00F000EEFEF0EE5003E09D
:103DC00003EC01F0FBD7200E03EC01F0480E03ECEE
:103DD00001F07A0E03EC01F00D0E03EC01F00A0E77
:103DE00003EC01F000EEFEF081EC00F00101A06FA9
:103DF00012C0A1F1A151A0110001D8A404EF1FF03D
:103E00000101A16B010EA06F0001130E0101A15D64
:103E10000001D8A01BEF1FF0D8A416EF1FF0890EE9
:103E20000101A05D0001D8A01BEF1FF0030E0101EE
:103E3000A16FE80EA06F00011200090EF76E460E8A
:103E4000F66EFBEC00F000EEFEF0EE5003E003EC4B
:103E500001F0FBD7200E03EC01F06D0E03EC01F036
:103E6000730E03EC01F02E0E03EC01F00D0E03ECCB
:103E700001F00A0E03EC01F000EEFEF081EC00F020
:103E80000101A26F12C0A3F1A351A2110001D8A495
:103E90004EEF1FF00101A36B010EA26F0001130E84
:103EA0000101A35D0001D8A064EF1FF0D8A460EF6A
:103EB0001FF0890E0101A25D0001D8A064EF1FF080
:103EC0000101A36B010EA26F00011200090EF76E33
:103ED0006C0EF66EFBEC00F000EEFEF0EE5003E030
:103EE00003EC01F0FBD7200E03EC01F06D0E03ECA8
:103EF00001F0730E03EC01F02E0E03EC01F00D0E39
:103F000003EC01F00A0E03EC01F000EEFEF081EC90
:103F100000F00101A46F12C0A5F1A551A411000188
:103F2000D8A497EF1FF00101A56B010EA46F00014B
:103F3000130E0101A55D0001D8A0ADEF1FF0D8A4BC
:103F4000A9EF1FF0890E0101A45D0001D8A0ADEF1B
:103F50001FF00101A56B010EA46F00011200090EF4
:103F6000F76E920EF66EFBEC00F000EEFEF0EE50F7
:103F700003E003EC01F0FBD7200E03EC01F06D0E23
:103F800003EC01F0730E03EC01F02E0E03EC01F0D4
:103F90000D0E03EC01F00A0E03EC01F000EEFEF052
:103FA00081EC00F00101A66F12C0A7F1A751A61184
:103FB0000001D8A4E0EF1FF00101A76B010EA66F6E
:103FC0000001130E0101A75D0001D8A0F6EF1FF05C
:103FD000D8A4F2EF1FF0890E0101A65D0001D8A060
:103FE000F6EF1FF00101A76B010EA66F0001120092
:103FF000090EF76EB80EF66EFBEC00F000EEFEF068
:10400000EE5003E003EC01F0FBD7200E03EC01F0CF
:104010006D0E03EC01F0730E03EC01F02E0E03ECB9
:1040200001F00D0E03EC01F00A0E03EC01F000EEBE
:10403000FEF081EC00F00101A86F12C0A9F1A951B6
:10404000A8110001D8A429EF20F00101A96B010EED
:10405000A86F0001130E0101A95D0001D8A03FEF78
:1040600020F0D8A43BEF20F0890E0101A85D0001EB
:10407000D8A03FEF20F00101A96B010EA86F00014D
:104080001200090EF76EDE0EF66EFBEC00F000EE8D
:10409000FEF0EE5003E003EC01F0FBD7200E03EC42
:1040A00001F06D0E03EC01F0730E03EC01F02E0E27
:1040B00003EC01F00D0E03EC01F00A0E03EC01F02D
:1040C00000EEFEF081EC00F00101AA6F12C0ABF12E
:1040D000AB51AA110001D8A472EF20F00101AB6B23
:1040E000010EAA6F0001130E0101AB5D0001D8A003
:1040F00088EF20F0D8A484EF20F0890E0101AA5D9A
:104100000001D8A088EF20F00101AB6B010EAA6F6F
:10411000000112000A0EF76E040EF66EFBEC00F0C2
:1041200000EEFEF0EE5003E003EC01F0FBD7200EB2
:1041300003EC01F06D0E03EC01F0730E03EC01F0E3
:104140002E0E03EC01F00D0E03EC01F00A0E03EC51
:1041500001F000EEFEF081EC00F00101AC6F12C046
:10416000ADF1AD51AC110001D8A4BBEF20F00101BD
:10417000AD6B010EAC6F0001130E0101AD5D0001CE
:10418000D8A0D1EF20F0D8A4CDEF20F0890E010106
:10419000AC5D0001D8A0D1EF20F00101AD6B010EA4
:1041A000AC6F000112000A0EF76E2A0EF66EFBECE1
:1041B00000F000EEFEF0EE5003E003EC01F0FBD760
:1041C000200E03EC01F06D0E03EC01F0730E03EC16
:1041D00001F02E0E03EC01F00D0E03EC01F00A0EBF
:1041E00003EC01F000EEFEF081EC00F00101AE6F97
:1041F00012C0AFF1AF51AE110001D8A404EF21F00D
:104200000101AF6B010EAE6F0001130E0101AF5D36
:104210000001D8A01AEF21F0D8A416EF21F0890EE2
:104220000101AE5D0001D8A01AEF21F00101AF6BD2
:10423000010EAE6F000112000A0EF76E500EF66E00
:10424000FBEC00F000EEFEF0EE5003E003EC01F0BA
:10425000FBD7200E03EC01F06D0E03EC01F0730EA2
:1042600003EC01F02E0E03EC01F00D0E03EC01F057
:104270000A0E03EC01F000EEFEF081EC00F001010B
:10428000B06F12C0B1F1B151B0110001D8A44DEF1F
:1042900021F00101B16B010EB06F0001130E01019D
:1042A000B15D0001D8A063EF21F0D8A45FEF21F049
:1042B000890E0101B05D0001D8A063EF21F001017A
:1042C000B16B010EB06F000112000A0EF76E760E90
:1042D000F66EFBEC00F000EEFEF0EE5003E003ECB7
:1042E00001F0FBD7200E03EC01F06D0E03EC01F0A2
:1042F000730E03EC01F02E0E03EC01F00D0E03EC37
:1043000001F00A0E03EC01F000EEFEF081EC00F08B
:104310000101B26F12C0B3F1B351B2110001D8A4C0
:1043200096EF21F00101B36B010EB26F0001130E85
:104330000101B35D0001D8A0ACEF21F0D8A4A8EF33
:1043400021F0890E0101B25D0001D8A0ACEF21F08F
:104350000101B36B010EB26F000112000A0EF76E7D
:104360009C0EF66EFBEC00F000EEFEF0EE5003E06B
:1043700003EC01F0FBD7200E03EC01F06D0E03EC13
:1043800001F0730E03EC01F02E0E03EC01F00D0EA4
:1043900003EC01F00A0E03EC01F000EEFEF081ECFC
:1043A00000F00101B46F12C0B5F1B551B4110001B4
:1043B000D8A4DFEF21F00101B56B010EB46F00014D
:1043C000130E0101B55D0001D8A0F5EF21F0D8A4CE
:1043D000F1EF21F0890E0101B45D0001D8A0F5EFE5
:1043E00021F00101B56B010EB46F000112000A0E3D
:1043F000F76ED80EF66EFBEC00F000EEFEF0EE501D
:1044000003E003EC01F0FBD7200E03EC01F06D0E8E
:1044100003EC01F0730E03EC01F02E0E03EC01F03F
:104420000D0E03EC01F00A0E03EC01F000EEFEF0BD
:1044300081EC00F00101746F12C075F175517411B7
:104440000001D8A428EF22F00101756B010E746FF2
:104450000001130E0101755D0001D8A03EEF22F0AE
:10446000D8A43AEF22F0890E0101745D0001D8A0B2
:104470003EEF22F00101756B010E746F0001120016
:104480000B0EF76E040EF66EFBEC00F000EEFEF085
:10449000EE5003E003EC01F0FBD7200E03EC01F03B
:1044A0006D0E03EC01F0730E03EC01F02E0E03EC25
:1044B00001F00D0E03EC01F00A0E03EC01F000EE2A
:1044C000FEF081EC00F00101946F12C095F195515E
:1044D00094110001D8A471EF22F00101956B010E37
:1044E000946F0001130E0101955D0001D8A087EFC4
:1044F00022F0D8A483EF22F0890E0101945D00011F
:10450000D8A087EF22F00101956B010E946F000196
:1045100012000B0EF76E300EF66EFBEC00F000EEA4
:10452000FEF0EE5003E003EC01F0FBD7200E03ECAD
:1045300001F06D0E03EC01F0730E03EC01F02E0E92
:1045400003EC01F00D0E03EC01F00A0E03EC01F098
:1045500000EEFEF081EC00F00101966F12C097F1C1
:10456000975196110001D8A4BAEF22F00101976B80
:10457000010E966F0001130E0101975D0001D8A096
:10458000D0EF22F0D8A4CCEF22F0890E0101965D85
:104590000001D8A0D0EF22F00101976B010E966FB9
:1045A000000112000B0EF76E560EF66EFBEC00F0DB
:1045B00000EEFEF0EE5003E003EC01F0FBD7200E1E
:1045C00003EC01F06D0E03EC01F0730E03EC01F04F
:1045D0002E0E03EC01F00D0E03EC01F00A0E03ECBD
:1045E00001F000EEFEF081EC00F00101B66F12C0A8
:1045F000B7F1B751B6110001D8A403EF23F00101C0
:10460000B76B010EB66F0001130E0101B75D00011B
:10461000D8A019EF23F0D8A415EF23F0890E0101DB
:10462000B65D0001D8A019EF23F00101B76B010EB0
:10463000B66F000112000B0EF76E7C0EF66EFBECEF
:1046400000F000EEFEF0EE5003E003EC01F0FBD7CB
:10465000200E03EC01F06D0E03EC01F0730E03EC81
:1046600001F02E0E03EC01F00D0E03EC01F00A0E2A
:1046700003EC01F000EEFEF081EC00F00101BA6FF6
:10468000820E026E040E076E9C0E046E400E036EC8
:10469000030E126EE80E116E31EC00F000011200F4
:1046A0000B0EF76E900EF66EFBEC00F000EEFEF0D7
:1046B00081EC00F00101686F0B0EF76EB20EF66E22
:1046C00000EEFEF097EC01F00001D8A47EEF23F09D
:1046D00001016D8B6D8D6D8FB881B883B885360EF5
:1046E00003EC01F0370E03EC01F02E0E03EC01F0A9
:1046F000300E03EC01F00001E8EF29F00B0EF76E2D
:10470000B60EF66E00EEFEF097EC01F0D8A49FEF27
:1047100023F001016D8B6D8D6D8FB891B893B885C5
:10472000360E03EC01F0390E03EC01F02E0E03EC13
:1047300001F0330E03EC01F00001E8EF29F00B0E5D
:10474000F76EBA0EF66E00EEFEF097EC01F0D8A40C
:10475000C0EF23F001016D9B6D8D6D8FB881B88323
:10476000B885370E03EC01F0310E03EC01F02E0E8C
:1047700003EC01F0390E03EC01F00001E8EF29F041
:104780000B0EF76EBE0EF66E00EEFEF097EC01F02B
:10479000D8A4E1EF23F001016D8B6D8D6D8FB88191
:1047A000B883B895370E03EC01F0340E03EC01F03A
:1047B0002E0E03EC01F0340E03EC01F00001E8EFE3
:1047C00029F00B0EF76EC20EF66E00EEFEF097ECBF
:1047D00001F0D8A401EF24F001016D9B6D9D6D8F58
:1047E000B881B883B885370E03EC01F003EC01F013
:1047F0002E0E03EC01F0300E03EC01F00001E8EFA7
:1048000029F00B0EF76EC60EF66E00EEFEF097EC7A
:1048100001F0D8A422EF24F001016D8B6D8D6D8F16
:10482000B881B893B885370E03EC01F0390E03EC6C
:1048300001F02E0E03EC01F0370E03EC01F0000145
:10484000E8EF29F00B0EF76ECA0EF66E00EEFEF0E2
:1048500097EC01F0D8A443EF24F001016D9B6D8D1E
:104860006D8FB881B883B895380E03EC01F0320E25
:1048700003EC01F02E0E03EC01F0350E03EC01F019
:104880000001E8EF29F00B0EF76ECE0EF66E00EE8B
:10489000FEF097EC01F0D8A464EF24F001016D8BD9
:1048A0006D8D6D8FB881B893B895380E03EC01F01B
:1048B000350E03EC01F02E0E03EC01F0340E03EC88
:1048C00001F00001E8EF29F00B0EF76ED20EF66E44
:1048D00000EEFEF097EC01F0D8A484EF24F0010183
:1048E0006D9B6D9D6D8FB881B883B895380E03ECC4
:1048F00001F003EC01F02E0E03EC01F0350E03EC99
:1049000001F00001E8EF29F00B0EF76ED60EF66EFF
:1049100000EEFEF097EC01F0D8A4A5EF24F0010121
:104920006D8B6D8D6D8FB891B883B885390E03ECA2
:1049300001F0310E03EC01F02E0E03EC01F0350E08
:1049400003EC01F00001E8EF29F00B0EF76EDA0E30
:10495000F66E00EEFEF097EC01F0D8A4C6EF24F05E
:1049600001016D9B6D8D6D8FB881B893B885390E3F
:1049700003EC01F0340E03EC01F02E0E03EC01F019
:10498000380E03EC01F00001E8EF29F00B0EF76E92
:10499000DE0EF66E00EEFEF097EC01F0D8A4E7EF25
:1049A00024F001016D8B6D8D6D8FB891B883B89532
:1049B000390E03EC01F0370E03EC01F02E0E03EC80
:1049C00001F0340E03EC01F00001E8EF29F00B0ECA
:1049D000F76EE20EF66E00EEFEF097EC01F0D8A452
:1049E0000AEF25F001016D9B6D9D6D8FB881B89325
:1049F000B885310E03EC01F0300E03EC01F003EC4E
:104A000001F02E0E03EC01F0300E03EC01F000017A
:104A1000E8EF29F00B0EF76EE60EF66E00EEFEF0F4
:104A200097EC01F0D8A42EEF25F001016D9B6D8D60
:104A30006D8FB881B893B895310E03EC01F0300E4C
:104A400003EC01F0330E03EC01F02E0E03EC01F049
:104A5000350E03EC01F00001E8EF29F00B0EF76EC4
:104A6000EA0EF66E00EEFEF097EC01F0D8A452EFDD
:104A700025F001016D9B6D9D6D8FB881B893B89540
:104A8000310E03EC01F0300E03EC01F0370E03ECB5
:104A900001F02E0E03EC01F0320E03EC01F00001E8
:104AA000E8EF29F00B0EF76EEE0EF66E00EEFEF05C
:104AB00097EC01F0D8A475EF25F001016D9B6D8D89
:104AC0006D8FB891B883B885310E03EC01F003EC1B
:104AD00001F0300E03EC01F02E0E03EC01F0390E64
:104AE00003EC01F00001E8EF29F00B0EF76EF20E77
:104AF000F66E00EEFEF097EC01F0D8A498EF25F0EA
:104B000001016D9B6D9D6D8FB891B883B885310E95
:104B100003EC01F003EC01F0340E03EC01F02E0E77
:104B200003EC01F0380E03EC01F00001E8EF29F08E
:104B30000B0EF76EF60EF66E00EEFEF097EC01F03F
:104B4000D8A4BBEF25F001016D9B6D8D6D8FB891E1
:104B5000B883B895310E03EC01F003EC01F0380E88
:104B600003EC01F02E0E03EC01F0380E03EC01F023
:104B70000001E8EF29F00B0EF76EFA0EF66E00EE6C
:104B8000FEF097EC01F0D8A4DFEF25F001016D9B5A
:104B90006D9D6D8FB891B883B895310E03EC01F01F
:104BA000320E03EC01F0330E03EC01F02E0E03EC99
:104BB00001F0300E03EC01F00001E8EF29F00B0EDC
:104BC000F76EFE0EF66E00EEFEF097EC01F0D8A444
:104BD00003EF26F001016D9B6D8D6D8FB891B89339
:104BE000B885310E03EC01F0320E03EC01F0370E04
:104BF00003EC01F02E0E03EC01F0330E03EC01F098
:104C00000001E8EF29F00C0EF76E020EF66E00EED2
:104C1000FEF097EC01F0D8A427EF26F001016D9B80
:104C20006D9D6D8FB891B893B885310E03EC01F08E
:104C3000330E03EC01F0310E03EC01F02E0E03EC09
:104C400001F0380E03EC01F00001E8EF29F00C0E42
:104C5000F76E060EF66E00EEFEF097EC01F0D8A4AB
:104C60004BEF26F001016D9B6D8D6D8FB891B89360
:104C7000B895310E03EC01F0330E03EC01F0360E63
:104C800003EC01F02E0E03EC01F0350E03EC01F005
:104C90000001E8EF29F00C0EF76E0A0EF66E00EE3A
:104CA000FEF097EC01F0D8A46FEF26F001016D9BA8
:104CB0006D9D6D8FB891B893B895310E03EC01F0EE
:104CC000340E03EC01F0310E03EC01F02E0E03EC78
:104CD00001F0330E03EC01F00001E8EF29F00C0EB7
:104CE000F76E0E0EF66E00EEFEF097EC01F0D8A413
:104CF00093EF26F001016D9B6D8D6D9FB881B88398
:104D0000B885310E03EC01F0340E03EC01F0360EE1
:104D100003EC01F02E0E03EC01F0320E03EC01F077
:104D20000001E8EF29F00C0EF76E120EF66E00EEA1
:104D3000FEF097EC01F0D8A4B7EF26F001016D9BCF
:104D40006D9D6D9FB881B883B885310E03EC01F07D
:104D5000350E03EC01F0310E03EC01F02E0E03ECE6
:104D600001F0340E03EC01F00001E8EF29F00C0E25
:104D7000F76E160EF66E00EEFEF097EC01F0D8A47A
:104D8000DBEF26F001016D9B6D8D6D9FB881B883BF
:104D9000B895310E03EC01F0350E03EC01F0360E40
:104DA00003EC01F02E0E03EC01F0370E03EC01F0E2
:104DB0000001E8EF29F00C0EF76E1A0EF66E00EE09
:104DC000FEF097EC01F0D8A4FFEF26F001016D8B07
:104DD0006D8D6D9FB891B893B885310E03EC01F0DD
:104DE000350E03EC01F0390E03EC01F02E0E03EC4E
:104DF00001F0380E03EC01F00001E8EF29F00C0E91
:104E0000F76E1E0EF66E00EEFEF097EC01F0D8A4E1
:104E100023EF27F001016D9B6D9D6D9FB881B883D5
:104E2000B895310E03EC01F0360E03EC01F0320EB2
:104E300003EC01F02E0E03EC01F0320E03EC01F056
:104E40000001E8EF29F00C0EF76E220EF66E00EE70
:104E5000FEF097EC01F0D8A447EF27F001016D9B1D
:104E60006D8D6D9FB881B893B885310E03EC01F05C
:104E7000360E03EC01F0370E03EC01F02E0E03ECBE
:104E800001F0390E03EC01F00001E8EF29F00C0EFF
:104E9000F76E260EF66E00EEFEF097EC01F0D8A449
:104EA0006BEF27F001016D9B6D9D6D9FB881B893ED
:104EB000B885310E03EC01F0370E03EC01F0330E30
:104EC00003EC01F02E0E03EC01F0380E03EC01F0C0
:104ED0000001E8EF29F00C0EF76E2A0EF66E00EED8
:104EE000FEF097EC01F0D8A48FEF27F001016D9B45
:104EF0006D8D6D9FB881B893B895310E03EC01F0BC
:104F0000370E03EC01F0390E03EC01F02E0E03EC2A
:104F100001F0390E03EC01F00001E8EF29F00C0E6E
:104F2000F76E2E0EF66E00EEFEF097EC01F0D8A4B0
:104F3000B3EF27F001016D8B6D8D6D9FB891B88334
:104F4000B895310E03EC01F0380E03EC01F0330E8E
:104F500003EC01F02E0E03EC01F0350E03EC01F032
:104F60000001E8EF29F00C0EF76E320EF66E00EE3F
:104F7000FEF097EC01F0D8A4D7EF27F001016D9B6C
:104F80006D9D6D9FB881B893B895310E03EC01F01B
:104F9000380E03EC01F0360E03EC01F02E0E03EC9C
:104FA00001F0320E03EC01F00001E8EF29F00C0EE5
:104FB000F76E360EF66E00EEFEF097EC01F0D8A418
:104FC000FBEF27F001016D8B6D8D6D9FB891B8835C
:104FD000B895310E03EC01F0380E03EC01F0390EF8
:104FE00003EC01F02E0E03EC01F0390E03EC01F09E
:104FF0000001E8EF29F00C0EF76E3A0EF66E00EEA7
:10500000FEF097EC01F0D8A41FEF28F001016D9B92
:105010006D8D6D9FB891B883B885310E03EC01F0AA
:10502000390E03EC01F0320E03EC01F02E0E03EC0E
:1050300001F0380E03EC01F00001E8EF29F00C0E4E
:10504000F76E3E0EF66E00EEFEF097EC01F0D8A47F
:1050500043EF28F001016D8B6D8D6D9FB881B89382
:10506000B895310E03EC01F0390E03EC01F0360E69
:1050700003EC01F02E0E03EC01F0360E03EC01F010
:105080000001E8EF29F00C0EF76E420EF66E00EE0E
:10509000FEF097EC01F0D8A466EF28F001016D8BCB
:1050A0006D8D6D9FB881B893B885310E03EC01F01A
:1050B000390E03EC01F003EC01F02E0E03EC01F0CD
:1050C000350E03EC01F00001E8EF29F00C0EF76E4D
:1050D000460EF66E00EEFEF097EC01F0D8A48AEFD3
:1050E00028F001016D9B6D9D6D9FB891B883B885C7
:1050F000320E03EC01F0300E03EC01F0330E03EC42
:1051000001F02E0E03EC01F0350E03EC01F000016E
:10511000E8EF29F00C0EF76E4A0EF66E00EEFEF088
:1051200097EC01F0D8A4AEEF28F001016D8B6D8DE6
:105130006D9FB881B883B895320E03EC01F0300E44
:1051400003EC01F0360E03EC01F02E0E03EC01F03F
:10515000350E03EC01F00001E8EF29F00C0EF76EBC
:105160004E0EF66E00EEFEF097EC01F0D8A4D2EFF2
:1051700028F001016D9B6D8D6D9FB891B883B89536
:10518000320E03EC01F0310E03EC01F0300E03ECB3
:1051900001F02E0E03EC01F0370E03EC01F00001DC
:1051A000E8EF29F00C0EF76E520EF66E00EEFEF0F0
:1051B00097EC01F0D8A4F6EF28F001016D9B6D9DEE
:1051C0006D9FB891B883B895320E03EC01F0310EA3
:1051D00003EC01F0380E03EC01F02E0E03EC01F0AD
:1051E000310E03EC01F00001E8EF29F00C0EF76E30
:1051F000560EF66E00EEFEF097EC01F0D8A419EF13
:1052000029F001016D9B6D8D6D9FB891B893B885A4
:10521000320E03EC01F003EC01F0350E03EC01F06B
:105220002E0E03EC01F0370E03EC01F00001E8EF65
:1052300029F00C0EF76E5A0EF66E00EEFEF097ECAB
:1052400001F0D8A43CEF29F001016D8B6D8D6D9FAD
:10525000B881B883B885320E03EC01F003EC01F09D
:10526000390E03EC01F02E0E03EC01F0310E03ECCD
:1052700001F00001E8EF29F00C0EF76E5E0EF66EFD
:1052800000EEFEF097EC01F0D8A45FEF29F00101E9
:105290006D9B6D9D6D9FB891B893B885320E03ECF0
:1052A00001F0330E03EC01F003EC01F02E0E03ECE1
:1052B00001F0360E03EC01F00001E8EF29F00C0ECE
:1052C000F76E620EF66E00EEFEF097EC01F0D8A4D9
:1052D00083EF29F001016D9B6D8D6D9FB891B8939F
:1052E000B895320E03EC01F0340E03EC01F0310EF0
:1052F00003EC01F02E0E03EC01F0380E03EC01F08C
:105300000001E8EF29F00C0EF76E660EF66E00EE67
:10531000FEF097EC01F0D8A4A7EF29F001016D9BF6
:105320006D9D6D9FB891B893B895320E03EC01F066
:10533000350E03EC01F0300E03EC01F02E0E03EC01
:1053400001F0330E03EC01F00001E8EF29F00C0E40
:10535000F76E6A0EF66E00EEFEF097EC01F0D8A440
:10536000CBEF29F001016D8B6D8D6D8FB891B893E6
:10537000B895320E03EC01F0350E03EC01F0340E5B
:1053800003EC01F02E0E03EC01F0310E03EC01F002
:105390000001E8EF29F0300EFE5DD8A4DDEF29F022
:1053A00001016D8B6D8D6D9FB891B893B895300EDE
:1053B00003EC01F00001E7EF29F001016D8B6D8D29
:1053C0006D9FB891B893B895300E03EC01F00001D1
:1053D000200E03EC01F0480E03EC01F07A0E03EC12
:1053E00001F00D0E03EC01F00A0E03EC01F0D8966B
:1053F0000101B8A7D8860001D8B6A1EF2AF0610E46
:1054000003EC01F0720E03EC01F0670E03EC01F007
:105410003D0E03EC01F000EEFEF0EE5003E003EC75
:1054200001F0FBD70D0E03EC01F00A0E03EC01F0C6
:1054300000EEFEF081EC00F00101686F0C0EF76EDB
:105440006E0EF66EFBEC00F0040E016E6851C9ECB6
:1054500000F00D0E03EC01F00A0E03EC01F00C0E4F
:10546000F76E7A0EF66EFBEC00F0040E016EE86A41
:105470006DBB010EC9EC00F00D0E03EC01F00A0E3D
:1054800003EC01F00C0EF76E860EF66EFBEC00F0EE
:10549000040E016EE86A6DBD010EC9EC00F00D0E40
:1054A00003EC01F00A0E03EC01F00C0EF76E920E05
:1054B000F66EFBEC00F0040E016EE86A6DBF010EA3
:1054C000C9EC00F00D0E03EC01F00A0E03EC01F044
:1054D0000C0EF76E9E0EF66EFBEC00F0040E016EE5
:1054E000E86AB8B1010EC9EC00F00D0E03EC01F052
:1054F0000A0E03EC01F00C0EF76EAA0EF66EFBEC32
:1055000000F0040E016EE86AB8B3010EC9EC00F0B9
:105510000D0E03EC01F00A0E03EC01F00C0EF76E19
:10552000B60EF66EFBEC00F0040E016EE86AB8B53C
:10553000010EC9EC00F00D0E03EC01F00A0E03ECB5
:1055400001F00001D89601016DABD8860001D8B6F4
:10555000AEEF2AF0929A808AB0EF2AF0929A809A5F
:10556000D89601016DADD8860001D8B6BCEF2AF0FF
:1055700092988088BEEF2AF092988098D896010180
:105580006DAFD8860001D8B6CAEF2AF09296808611
:10559000CCEF2AF092968096D8960101B8A1D886D1
:1055A0000001D8B6D8EF2AF092948084DAEF2AF07E
:1055B00092948094D8960101B8A3D8860001D8B6F9
:1055C000E6EF2AF092928082E8EF2AF0929280929F
:1055D000D8960101B8A5D8860001D8B6F4EF2AF014
:1055E00092908080F6EF2AF0929080901200D896E8
:1055F0000101B8A7D8860001D8B611EF2BF00C0E28
:10560000F76EC20EF66EFBEC00F0040E016E0101A7
:105610006851C9EC00F00D0E03EC01F00A0E03EC2A
:1056200001F000010D0E03EC01F00A0E03EC01F095
:10563000140E2CEC01F0AA6AA96A010168511EEC53
:1056400001F00C0EF76EDA0EF66EFBEC00F0040EB5
:10565000016E6851C9EC00F00D0E03EC01F00A0E6A
:1056600003EC01F00A0E2CEC01F0AA6A010EA96EFF
:105670006B511EEC01F06C511EEC01F00C0EF76E3C
:10568000F20EF66EFBEC00F00D0E03EC01F00A0ECC
:1056900003EC01F0AA6A030EA96E6E511EEC01F034
:1056A0006F511EEC01F00D0EF76E0A0EF66EFBEC5C
:1056B00000F00D0E03EC01F00A0E03EC01F0AA6AF3
:1056C000050EA96E74511EEC01F075511EEC01F02F
:1056D0000D0EF76E220EF66EFBEC00F00D0E03ECD5
:1056E00001F00A0E03EC01F0AA6A070EA96E7651CA
:1056F0001EEC01F077511EEC01F00D0EF76E3E0E20
:10570000F66EFBEC00F00D0E03EC01F00A0E03EC5C
:1057100001F0AA6A090EA96E80511EEC01F08151B8
:105720001EEC01F00D0EF76E5A0EF66EFBEC00F05B
:105730000D0E03EC01F00A0E03EC01F0AA6A0B0E49
:10574000A96E8A511EEC01F08B511EEC01F00D0E7A
:10575000F76E740EF66EFBEC00F00D0E03EC01F02C
:105760000A0E03EC01F0AA6A0D0EA96E78511EEC28
:1057700001F079511EEC01F00D0EF76E8C0EF66EF5
:10578000FBEC00F00D0E03EC01F00A0E03EC01F04F
:10579000AA6A0F0EA96E82511EEC01F083511EEC15
:1057A00001F00D0EF76EA80EF66EFBEC00F00D0E7C
:1057B00003EC01F00A0E03EC01F0AA6A110EA96EC7
:1057C0008C511EEC01F08D511EEC01F00D0EF76EA8
:1057D000C20EF66EFBEC00F00D0E03EC01F00A0EAB
:1057E00003EC01F0AA6A130EA96E7A511EEC01F0C7
:1057F0007B511EEC01F00D0EF76EDA0EF66EFBEC2F
:1058000000F00D0E03EC01F00A0E03EC01F0AA6AA1
:10581000150EA96E84511EEC01F085511EEC01F0AD
:105820000D0EF76EF60EF66EFBEC00F00D0E03ECAF
:1058300001F00A0E03EC01F0AA6A170EA96E8E5150
:105840001EEC01F08F511EEC01F00E0EF76E100EE3
:10585000F66EFBEC00F00D0E03EC01F00A0E03EC0B
:1058600001F0AA6A190EA96E7C511EEC01F07D515F
:105870001EEC01F00E0EF76E280EF66EFBEC00F03B
:105880000D0E03EC01F00A0E03EC01F0AA6A1B0EE8
:10589000A96E86511EEC01F087511EEC01F00E0E30
:1058A000F76E440EF66EFBEC00F00D0E03EC01F00B
:1058B0000A0E03EC01F0AA6A1D0EA96E90511EECAF
:1058C00001F091511EEC01F00E0EF76E5E0EF66EB9
:1058D000FBEC00F00D0E03EC01F00A0E03EC01F0FE
:1058E000AA6A1F0EA96E7E511EEC01F07F511EECBC
:1058F00001F00E0EF76E760EF66EFBEC00F00D0E5C
:1059000003EC01F00A0E03EC01F0AA6A210EA96E65
:1059100088511EEC01F089511EEC01F00E0EF76E5D
:10592000920EF66EFBEC00F00D0E03EC01F00A0E89
:1059300003EC01F0AA6A230EA96E92511EEC01F04D
:1059400093511EEC01F00E0EF76EAC0EF66EFBECF2
:1059500000F00D0E03EC01F00A0E03EC01F0AA6A50
:10596000250EA96E94511EEC01F095511EEC01F02C
:105970000E0EF76EC40EF66EFBEC00F00D0E03EC8F
:1059800001F00A0E03EC01F0AA6A270EA96E9651E7
:105990001EEC01F097511EEC01F00E0EF76EE00EBA
:1059A000F66EFBEC00F00D0E03EC01F00A0E03ECBA
:1059B00001F0AA6A290EA96E98511EEC01F09951C6
:1059C0001EEC01F00E0EF76EFC0EF66EFBEC00F016
:1059D0000D0E03EC01F00A0E03EC01F0AA6A2B0E87
:1059E000A96EA2511EEC01F0A3511EEC01F00F0EA6
:1059F000F76E180EF66EFBEC00F00D0E03EC01F0E6
:105A00000A0E03EC01F0AA6A2D0EA96EAC511EEC31
:105A100001F0AD511EEC01F00F0EF76E320EF66E76
:105A2000FBEC00F00D0E03EC01F00A0E03EC01F0AC
:105A3000AA6A2F0EA96E9A511EEC01F09B511EEC22
:105A400001F00F0EF76E4A0EF66EFBEC00F00D0E35
:105A500003EC01F00A0E03EC01F0AA6A310EA96E04
:105A6000A4511EEC01F0A5511EEC01F00F0EF76ED3
:105A7000660EF66EFBEC00F00D0E03EC01F00A0E64
:105A800003EC01F0AA6A330EA96EAE511EEC01F0D0
:105A9000AF511EEC01F00F0EF76E800EF66EFBECB0
:105AA00000F00D0E03EC01F00A0E03EC01F0AA6AFF
:105AB000350EA96E9C511EEC01F09D511EEC01F0BB
:105AC0000F0EF76E980EF66EFBEC00F00D0E03EC69
:105AD00001F00A0E03EC01F0AA6A370EA96EA65176
:105AE0001EEC01F0A7511EEC01F00F0EF76EB40E84
:105AF000F66EFBEC00F00D0E03EC01F00A0E03EC69
:105B000001F0AA6A390EA96EB0511EEC01F0B15134
:105B10001EEC01F00F0EF76ECE0EF66EFBEC00F0F1
:105B20000D0E03EC01F00A0E03EC01F0AA6A3B0E25
:105B3000A96E9E511EEC01F09F511EEC01F00F0E5C
:105B4000F76EE60EF66EFBEC00F00D0E03EC01F0C6
:105B50000A0E03EC01F0AA6A3D0EA96EA8511EECD4
:105B600001F0A9511EEC01F0100EF76E020EF66E58
:105B7000FBEC00F00D0E03EC01F00A0E03EC01F05B
:105B8000AA6A3F0EA96EB2511EEC01F0B3511EEC91
:105B900001F0100EF76E1C0EF66EFBEC00F00D0E11
:105BA00003EC01F00A0E03EC01F0AA6A410EA96EA3
:105BB000A0511EEC01F0A1511EEC01F0100EF76E89
:105BC000340EF66EFBEC00F00D0E03EC01F00A0E45
:105BD00003EC01F0AA6A430EA96EAA511EEC01F073
:105BE000AB511EEC01F0100EF76E500EF66EFBEC92
:105BF00000F00D0E03EC01F00A0E03EC01F0AA6AAE
:105C0000450EA96EB4511EEC01F0B5511EEC01F029
:105C1000100EF76E6A0EF66EFBEC00F00D0E03EC44
:105C200001F00A0E03EC01F0AA6A470EA96EB65104
:105C30001EEC01F0B7511EEC01F0100EF76E820E53
:105C4000F66EFBEC00F00D0E03EC01F00A0E03EC17
:105C500001F0100EF76E9E0EF66EFBEC00F00D0ECE
:105C600003EC01F00A0E03EC01F00D0E03EC01F061
:105C70000A0E03EC01F000011200100EF76EC40EC4
:105C8000F66EFBEC00F00D0E03EC01F00A0E03ECD7
:105C900001F0000E15EC01F00101686F010E15EC2A
:105CA00001F06B6F17EC01F06C6F030E15EC01F057
:105CB0006E6F17EC01F06F6F050E15EC01F0746F4D
:105CC00017EC01F0756F070E15EC01F0766F17EC0D
:105CD00001F0776F090E15EC01F0806F17EC01F001
:105CE000816F0B0E15EC01F08A6F17EC01F08B6FD2
:105CF0000D0E15EC01F0786F17EC01F0796F0F0EB7
:105D000015EC01F0826F17EC01F0836F110E15ECAA
:105D100001F08C6F17EC01F08D6F130E15EC01F094
:105D20007A6F17EC01F07B6F150E15EC01F0846FA4
:105D300017EC01F0856F170E15EC01F08E6F17EC64
:105D400001F08F6F190E15EC01F07C6F17EC01F06C
:105D50007D6F1B0E15EC01F0866F17EC01F0876F5D
:105D60001D0E15EC01F0906F17EC01F0916F1F0EF6
:105D700015EC01F07E6F17EC01F07F6F210E15EC32
:105D800001F0886F17EC01F0896F230E15EC01F01C
:105D9000926F17EC01F0936F250E15EC01F0946FE4
:105DA00017EC01F0956F270E15EC01F0966F17ECCC
:105DB00001F0976F290E15EC01F0986F17EC01F0C8
:105DC000996F2B0E15EC01F0A26F17EC01F0A36F89
:105DD0002D0E15EC01F0AC6F17EC01F0AD6F2F0E2E
:105DE00015EC01F09A6F17EC01F09B6F310E15EC7A
:105DF00001F0A46F17EC01F0A56F330E15EC01F064
:105E0000AE6F17EC01F0AF6F350E15EC01F09C6F23
:105E100017EC01F09D6F370E15EC01F0A66F17EC33
:105E200001F0A76F390E15EC01F0B06F17EC01F01F
:105E3000B16F3B0E15EC01F09E6F17EC01F09F6FF8
:105E40003D0E15EC01F0A86F17EC01F0A96F3F0EA5
:105E500015EC01F0B26F17EC01F0B36F410E15ECC9
:105E600001F0A06F17EC01F0A16F430E15EC01F0EB
:105E7000AA6F17EC01F0AB6F450E15EC01F0B46F93
:105E800017EC01F0B56F470E15EC01F0B66F17EC8B
:105E900001F0B76F100EF76EEC0EF66EFBEC00F033
:105EA0000D0E03EC01F00A0E03EC01F0D896B8A732
:105EB000D8860001D8B66FEF2FF0110EF76E060EE0
:105EC000F66EFBEC00F0040E016E01016851C9ECA6
:105ED00000F00D0E03EC01F00A0E03EC01F00001DE
:105EE000FB0E0101685D0001D8A079EF2FF00101E0
:105EF000686B0001D8960101B8A7D8860001D8B612
:105F000094EF2FF0110EF76E120EF66EFBEC00F010
:105F1000040E016E01016851C9EC00F00D0E03EC96
:105F200001F00A0E03EC01F0000100EEFEF0020E9B
:105F3000016E01016851C9EC00F0EF6AD896B8A76C
:105F4000D8860001D8B6B8EF2FF0110EF76E1E0EEE
:105F5000F66EFBEC00F000EEFEF0EE5003E003EC1A
:105F600001F0FBD70D0E03EC01F00A0E03EC01F07B
:105F700050EC23F0130E01016C5D0001D8A0CFEFAF
:105F80002FF0D8A4CBEF2FF0890E01016B5D00013B
:105F9000D8A0CFEF2FF001016C6B010E6B6F0001E9
:105FA000130E01016F5D0001D8A0E5EF2FF0D8A41A
:105FB000E1EF2FF0890E01016E5D0001D8A0E5EF41
:105FC0002FF001016F6B010E6E6F0001130E0101C6
:105FD000755D0001D8A0FBEF2FF0D8A4F7EF2FF0EC
:105FE000890E0101745D0001D8A0FBEF2FF00101C3
:105FF000756B010E746F0001130E0101775D0001D6
:10600000D8A011EF30F0D8A40DEF30F0890E0101C7
:10601000765D0001D8A011EF30F00101776B010E21
:10602000766F0001130E0101795D0001D8A027EF02
:1060300030F0D8A423EF30F0890E0101785D000123
:10604000D8A027EF30F00101796B010E786F0001C5
:10605000130E01017B5D0001D8A03DEF30F0D8A404
:1060600039EF30F0890E01017A5D0001D8A03DEFD3
:1060700030F001017B6B010E7A6F0001130E0101FC
:106080007D5D0001D8A053EF30F0D8A44FEF30F081
:10609000890E01017C5D0001D8A053EF30F00101B1
:1060A0007D6B010E7C6F0001130E01017F5D00010D
:1060B000D8A069EF30F0D8A465EF30F0890E010167
:1060C0007E5D0001D8A069EF30F001017F6B010E09
:1060D0007E6F0001130E0101815D0001D8A07FEFEA
:1060E00030F0D8A47BEF30F0890E0101805D000113
:1060F000D8A07FEF30F00101816B010E806F0001AD
:10610000130E0101835D0001D8A095EF30F0D8A4F3
:1061100091EF30F0890E0101825D0001D8A095EF6A
:1061200030F00101836B010E826F0001130E01013B
:10613000855D0001D8A0ABEF30F0D8A4A7EF30F018
:10614000890E0101845D0001D8A0ABEF30F00101A0
:10615000856B010E846F0001130E0101875D000144
:10616000D8A0C1EF30F0D8A4BDEF30F0890E010106
:10617000865D0001D8A0C1EF30F00101876B010EF0
:10618000866F0001130E0101895D0001D8A0D7EFD1
:1061900030F0D8A4D3EF30F0890E0101885D000102
:1061A000D8A0D7EF30F00101896B010E886F000194
:1061B000130E01018B5D0001D8A0EDEF30F0D8A4E3
:1061C000E9EF30F0890E01018A5D0001D8A0EDEF02
:1061D00030F001018B6B010E8A6F0001130E01017B
:1061E0008D5D0001D8A003EF31F0D8A4FFEF30F0AF
:1061F000890E01018C5D0001D8A003EF31F001018F
:106200008D6B010E8C6F0001130E01018F5D00017B
:10621000D8A019EF31F0D8A415EF31F0890E0101A3
:106220008E5D0001D8A019EF31F001018F6B010ED6
:106230008E6F0001130E0101915D0001D8A02FEFB8
:1062400031F0D8A42BEF31F0890E0101905D0001EF
:10625000D8A02FEF31F00101916B010E906F00017A
:10626000130E0101935D0001D8A045EF31F0D8A4D1
:1062700041EF31F0890E0101925D0001D8A045EF98
:1062800031F00101936B010E926F0001130E0101B9
:10629000955D0001D8A05BEF31F0D8A457EF31F045
:1062A000890E0101945D0001D8A05BEF31F001017E
:1062B000956B010E946F0001130E0101975D0001B3
:1062C000D8A071EF31F0D8A46DEF31F0890E010143
:1062D000965D0001D8A071EF31F00101976B010EBE
:1062E000966F0001130E0101995D0001D8A087EFA0
:1062F00031F0D8A483EF31F0890E0101985D0001DF
:10630000D8A087EF31F00101996B010E986F000161
:10631000130E01019B5D0001D8A09DEF31F0D8A4C0
:1063200099EF31F0890E01019A5D0001D8A09DEF2F
:1063300031F001019B6B010E9A6F0001130E0101F8
:106340009D5D0001D8A0B3EF31F0D8A4AFEF31F0DC
:10635000890E01019C5D0001D8A0B3EF31F001016D
:106360009D6B010E9C6F0001130E01019F5D0001EA
:10637000D8A0C9EF31F0D8A4C5EF31F0890E0101E2
:106380009E5D0001D8A0C9EF31F001019F6B010EA5
:106390009E6F0001130E0101A15D0001D8A0DFEF87
:1063A00031F0D8A4DBEF31F0890E0101A05D0001CE
:1063B000D8A0DFEF31F00101A16B010EA06F000149
:1063C000130E0101A35D0001D8A0F5EF31F0D8A4B0
:1063D000F1EF31F0890E0101A25D0001D8A0F5EFC7
:1063E00031F00101A36B010EA26F0001130E010138
:1063F000A55D0001D8A00BEF32F0D8A407EF32F072
:10640000890E0101A45D0001D8A00BEF32F001015B
:10641000A56B010EA46F0001130E0101A75D000121
:10642000D8A021EF32F0D8A41DEF32F0890E01017F
:10643000A65D0001D8A021EF32F00101A76B010E8B
:10644000A66F0001130E0101A95D0001D8A037EF6E
:1064500032F0D8A433EF32F0890E0101A85D0001BB
:10646000D8A037EF32F00101A96B010EA86F00012F
:10647000130E0101AB5D0001D8A04DEF32F0D8A49E
:1064800049EF32F0890E0101AA5D0001D8A04DEF5D
:1064900032F00101AB6B010EAA6F0001130E010176
:1064A000AD5D0001D8A063EF32F0D8A45FEF32F009
:1064B000890E0101AC5D0001D8A063EF32F001014B
:1064C000AD6B010EAC6F0001130E0101AF5D000159
:1064D000D8A079EF32F0D8A475EF32F0890E01011F
:1064E000AE5D0001D8A079EF32F00101AF6B010E73
:1064F000AE6F0001130E0101B15D0001D8A08FEF56
:1065000032F0D8A48BEF32F0890E0101B05D0001AA
:10651000D8A08FEF32F00101B16B010EB06F000116
:10652000130E0101B35D0001D8A0A5EF32F0D8A48D
:10653000A1EF32F0890E0101B25D0001D8A0A5EFF4
:1065400032F00101B36B010EB26F0001130E0101B5
:10655000B55D0001D8A0BBEF32F0D8A4B7EF32F0A0
:10656000890E0101B45D0001D8A0BBEF32F001013A
:10657000B56B010EB46F0001130E0101B75D000190
:10658000D8A0D1EF32F0D8A4CDEF32F0890E0101BE
:10659000B65D0001D8A0D1EF32F00101B76B010E5A
:1065A000B66F000101EEBCF0020E016E01016851F0
:1065B000C9EC00F0EF6A110EF76E260EF66EFBECDA
:1065C00000F001EEBCF0EE5003E003EC01F0FBD76D
:1065D0000D0E03EC01F00A0E03EC01F001EEBCF02D
:1065E000020E016E066A6CC112F06BC111F0CCECA8
:1065F00000F0EF6A110EF76E3A0EF66EFBEC00F04B
:1066000001EEBCF0EE5003E003EC01F0FBD70D0E01
:1066100003EC01F00A0E03EC01F001EEBCF0020EF7
:10662000016E066A6FC112F06EC111F0CCEC00F081
:10663000EF6A110EF76E500EF66EFBEC00F001EEF5
:10664000BCF0EE5003E003EC01F0FBD70D0E03ECC1
:1066500001F00A0E03EC01F001EEBCF0020E016E37
:10666000066A75C112F074C111F0CCEC00F0EF6A4B
:10667000110EF76E660EF66EFBEC00F001EEBCF04C
:10668000EE5003E003EC01F0FBD70D0E03EC01F03C
:106690000A0E03EC01F001EEBCF0020E016E066A78
:1066A00077C112F076C111F0CCEC00F0EF6A110E58
:1066B000F76E7C0EF66EFBEC00F001EEBCF0EE50D7
:1066C00003E003EC01F0FBD70D0E03EC01F00A0E22
:1066D00003EC01F001EEBCF0020E016E066A81C10E
:1066E00012F080C111F0CCEC00F0EF6A110EF76EE1
:1066F000980EF66EFBEC00F001EEBCF0EE5003E0FD
:1067000003EC01F0FBD70D0E03EC01F00A0E03ECD5
:1067100001F001EEBCF0020E016E066A8BC112F0B0
:106720008AC111F0CCEC00F0EF6A110EF76EB40ED6
:10673000F66EFBEC00F001EEBCF0EE5003E003EC73
:1067400001F0FBD70D0E03EC01F00A0E03EC01F093
:1067500001EEBCF0020E016E066A79C112F078C13A
:1067600011F0CCEC00F0EF6A110EF76ECA0EF66E67
:10677000FBEC00F001EEBCF0EE5003E003EC01F0A6
:10678000FBD70D0E03EC01F00A0E03EC01F001EE55
:10679000BCF0020E016E066A83C112F082C111F0D4
:1067A000CCEC00F0EF6A110EF76EE60EF66EFBEC25
:1067B00000F001EEBCF0EE5003E003EC01F0FBD77B
:1067C0000D0E03EC01F00A0E03EC01F001EEBCF03B
:1067D000020E016E066A8DC112F08CC111F0CCEC74
:1067E00000F0EF6A120EF76E020EF66EFBEC00F090
:1067F00001EEBCF0EE5003E003EC01F0FBD70D0E10
:1068000003EC01F00A0E03EC01F001EEBCF0020E05
:10681000016E066A7BC112F07AC111F0CCEC00F077
:10682000EF6A120EF76E180EF66EFBEC00F001EE3A
:10683000BCF0EE5003E003EC01F0FBD70D0E03ECCF
:1068400001F00A0E03EC01F001EEBCF0020E016E45
:10685000066A85C112F084C111F0CCEC00F0EF6A39
:10686000120EF76E340EF66EFBEC00F001EEBCF08B
:10687000EE5003E003EC01F0FBD70D0E03EC01F04A
:106880000A0E03EC01F001EEBCF0020E016E066A86
:106890008FC112F08EC111F0CCEC00F0EF6A120E35
:1068A000F76E500EF66EFBEC00F001EEBCF0EE5011
:1068B00003E003EC01F0FBD70D0E03EC01F00A0E30
:1068C00003EC01F001EEBCF0020E016E066A7DC120
:1068D00012F07CC111F0CCEC00F0EF6A120EF76EF2
:1068E000660EF66EFBEC00F001EEBCF0EE5003E03D
:1068F00003EC01F0FBD70D0E03EC01F00A0E03ECE4
:1069000001F001EEBCF0020E016E066A87C112F0C2
:1069100086C111F0CCEC00F0EF6A120EF76E820E19
:10692000F66EFBEC00F001EEBCF0EE5003E003EC81
:1069300001F0FBD70D0E03EC01F00A0E03EC01F0A1
:1069400001EEBCF0020E016E066A91C112F090C118
:1069500011F0CCEC00F0EF6A120EF76E9E0EF66EA0
:10696000FBEC00F001EEBCF0EE5003E003EC01F0B4
:10697000FBD70D0E03EC01F00A0E03EC01F001EE63
:10698000BCF0020E016E066A7FC112F07EC111F0EA
:10699000CCEC00F0EF6A120EF76EB40EF66EFBEC64
:1069A00000F001EEBCF0EE5003E003EC01F0FBD789
:1069B0000D0E03EC01F00A0E03EC01F001EEBCF049
:1069C000020E016E066A89C112F088C111F0CCEC8A
:1069D00000F0EF6A120EF76ED00EF66EFBEC00F0D0
:1069E00001EEBCF0EE5003E003EC01F0FBD70D0E1E
:1069F00003EC01F00A0E03EC01F001EEBCF0020E14
:106A0000016E066A93C112F092C111F0CCEC00F055
:106A1000EF6A120EF76EEC0EF66EFBEC00F001EE74
:106A2000BCF0EE5003E003EC01F0FBD70D0E03ECDD
:106A300001F00A0E03EC01F001EEBCF0020E016E53
:106A4000066A95C112F094C111F0CCEC00F0EF6A27
:106A5000130EF76E020EF66EFBEC00F001EEBCF0CA
:106A6000EE5003E003EC01F0FBD70D0E03EC01F058
:106A70000A0E03EC01F001EEBCF0020E016E066A94
:106A800097C112F096C111F0CCEC00F0EF6A130E32
:106A9000F76E180EF66EFBEC00F001EEBCF0EE5057
:106AA00003E003EC01F0FBD70D0E03EC01F00A0E3E
:106AB00003EC01F001EEBCF0020E016E066A99C112
:106AC00012F098C111F0CCEC00F0EF6A130EF76EE3
:106AD0002E0EF66EFBEC00F001EEBCF0EE5003E083
:106AE00003EC01F0FBD70D0E03EC01F00A0E03ECF2
:106AF00001F001EEBCF0020E016E066AA3C112F0B5
:106B0000A2C111F0CCEC00F0EF6A130EF76E4A0E42
:106B1000F66EFBEC00F001EEBCF0EE5003E003EC8F
:106B200001F0FBD70D0E03EC01F00A0E03EC01F0AF
:106B300001EEBCF0020E016E066AADC112F0ACC1EE
:106B400011F0CCEC00F0EF6A130EF76E660EF66EE5
:106B5000FBEC00F001EEBCF0EE5003E003EC01F0C2
:106B6000FBD70D0E03EC01F00A0E03EC01F001EE71
:106B7000BCF0020E016E066A9BC112F09AC111F0C0
:106B8000CCEC00F0EF6A130EF76E7C0EF66EFBECA9
:106B900000F001EEBCF0EE5003E003EC01F0FBD797
:106BA0000D0E03EC01F00A0E03EC01F001EEBCF057
:106BB000020E016E066AA5C112F0A4C111F0CCEC60
:106BC00000F0EF6A130EF76E980EF66EFBEC00F015
:106BD00001EEBCF0EE5003E003EC01F0FBD70D0E2C
:106BE00003EC01F00A0E03EC01F001EEBCF0020E22
:106BF000016E066AAFC112F0AEC111F0CCEC00F02C
:106C0000EF6A130EF76EB40EF66EFBEC00F001EEB9
:106C1000BCF0EE5003E003EC01F0FBD70D0E03ECEB
:106C200001F00A0E03EC01F001EEBCF0020E016E61
:106C3000066A9DC112F09CC111F0CCEC00F0EF6A25
:106C4000130EF76ECA0EF66EFBEC00F001EEBCF010
:106C5000EE5003E003EC01F0FBD70D0E03EC01F066
:106C60000A0E03EC01F001EEBCF0020E016E066AA2
:106C7000A7C112F0A6C111F0CCEC00F0EF6A130E20
:106C8000F76EE60EF66EFBEC00F001EEBCF0EE5097
:106C900003E003EC01F0FBD70D0E03EC01F00A0E4C
:106CA00003EC01F001EEBCF0020E016E066AB1C108
:106CB00012F0B0C111F0CCEC00F0EF6A140EF76ED8
:106CC000020EF66EFBEC00F001EEBCF0EE5003E0BD
:106CD00003EC01F0FBD70D0E03EC01F00A0E03EC00
:106CE00001F001EEBCF0020E016E066A9FC112F0C7
:106CF0009EC111F0CCEC00F0EF6A140EF76E180E86
:106D0000F66EFBEC00F001EEBCF0EE5003E003EC9D
:106D100001F0FBD70D0E03EC01F00A0E03EC01F0BD
:106D200001EEBCF0020E016E066AA9C112F0A8C104
:106D300011F0CCEC00F0EF6A140EF76E340EF66E24
:106D4000FBEC00F001EEBCF0EE5003E003EC01F0D0
:106D5000FBD70D0E03EC01F00A0E03EC01F001EE7F
:106D6000BCF0020E016E066AB3C112F0B2C111F09E
:106D7000CCEC00F0EF6A140EF76E500EF66EFBECE2
:106D800000F001EEBCF0EE5003E003EC01F0FBD7A5
:106D90000D0E03EC01F00A0E03EC01F001EEBCF065
:106DA000020E016E066AA1C112F0A0C111F0CCEC76
:106DB00000F0EF6A140EF76E660EF66EFBEC00F054
:106DC00001EEBCF0EE5003E003EC01F0FBD70D0E3A
:106DD00003EC01F00A0E03EC01F001EEBCF0020E30
:106DE000016E066AABC112F0AAC111F0CCEC00F042
:106DF000EF6A140EF76E820EF66EFBEC00F001EEF9
:106E0000BCF0EE5003E003EC01F0FBD70D0E03ECF9
:106E100001F00A0E03EC01F001EEBCF0020E016E6F
:106E2000066AB5C112F0B4C111F0CCEC00F0EF6A03
:106E3000140EF76E9E0EF66EFBEC00F001EEBCF049
:106E4000EE5003E003EC01F0FBD70D0E03EC01F074
:106E50000A0E03EC01F001EEBCF0020E016E066AB0
:106E6000B7C112F0B6C111F0CCEC00F0EF6A140E0D
:106E7000F76EB40EF66EFBEC00F001EEBCF0EE50D7
:106E800003E003EC01F0FBD70D0E03EC01F00A0E5A
:106E900003EC01F0140EF76ECA0EF66EFBEC00F078
:106EA0000D0E03EC01F00A0E03EC01F000011200DC
:106EB00094988288D8960101B8A7D8860001D8B6E0
:106EC00087EF37F001EEBCF0020E016E066A75C165
:106ED00012F074C111F0CCEC00F0EF6A0D0E03EC6F
:106EE00001F00A0E03EC01F0140EF76EE40EF66EDC
:106EF000FBEC00F001EEBCF0EE5003E003EC01F01F
:106F0000FBD70D0E03EC01F00A0E03EC01F075C186
:106F100010F0010174512DEC01F0D896B8A7D88675
:106F20000001D8B6B3EF37F001EEBCF0020E016EEF
:106F3000066A81C112F080C111F0CCEC00F0EF6A5A
:106F4000140EF76EF60EF66EFBEC00F001EEBCF0E0
:106F5000EE5003E003EC01F0FBD70D0E03EC01F063
:106F60000A0E03EC01F0D8960101B8A7D8860001FB
:106F7000D8B6DAEF37F001EEBCF0020E016E066A09
:106F800077C112F076C111F0CCEC00F0EF6A150E6B
:106F9000F76E080EF66EFBEC00F001EEBCF0EE5062
:106FA00003E003EC01F0FBD70D0E03EC01F00A0E39
:106FB00003EC01F0820E026E040E076E81C104F034
:106FC00080C103F077C112F076C111F031EC00F00E
:106FD000D8960101B8A7D8860001D8B60FEF38F0CF
:106FE00001EEBCF0020E016E066A8BC112F08AC17E
:106FF00011F0CCEC00F0EF6A150EF76E1A0EF66E7B
:10700000FBEC00F001EEBCF0EE5003E003EC01F00D
:10701000FBD70D0E03EC01F00A0E03EC01F08BC15F
:1070200010F001018A512DEC01F0D896B8A7D8864E
:107030000001D8B63BEF38F001EEBCF0020E016E55
:10704000066A83C112F082C111F0CCEC00F0EF6A45
:10705000150EF76E2C0EF66EFBEC00F001EEBCF098
:10706000EE5003E003EC01F0FBD70D0E03EC01F052
:107070000A0E03EC01F0D8960101B8A7D8860001EA
:10708000D8B662EF38F001EEBCF0020E016E066A6F
:1070900079C112F078C111F0CCEC00F0EF6A150E56
:1070A000F76E3E0EF66EFBEC00F001EEBCF0EE501B
:1070B00003E003EC01F0FBD70D0E03EC01F00A0E28
:1070C00003EC01F0820E026E040E076E83C104F021
:1070D00082C103F079C112F078C111F031EC00F0F7
:1070E000D8960101B8A7D8860001D8B697EF38F036
:1070F00001EEBCF0020E016E066A8DC112F08CC169
:1071000011F0CCEC00F0EF6A150EF76E500EF66E33
:10711000FBEC00F001EEBCF0EE5003E003EC01F0FC
:10712000FBD70D0E03EC01F00A0E03EC01F08DC14C
:1071300010F001018C512DEC01F0D896B8A7D8863B
:107140000001D8B6C3EF38F001EEBCF0020E016EBC
:10715000066A85C112F084C111F0CCEC00F0EF6A30
:10716000150EF76E620EF66EFBEC00F001EEBCF051
:10717000EE5003E003EC01F0FBD70D0E03EC01F041
:107180000A0E03EC01F0D8960101B8A7D8860001D9
:10719000D8B6EAEF38F001EEBCF0020E016E066AD6
:1071A0007BC112F07AC111F0CCEC00F0EF6A150E41
:1071B000F76E740EF66EFBEC00F001EEBCF0EE50D4
:1071C00003E003EC01F0FBD70D0E03EC01F00A0E17
:1071D00003EC01F0820E026E040E076E85C104F00E
:1071E00084C103F07BC112F07AC111F031EC00F0E0
:1071F000D8960101B8A7D8860001D8B61FEF39F09C
:1072000001EEBCF0020E016E066A8FC112F08EC153
:1072100011F0CCEC00F0EF6A150EF76E860EF66EEC
:10722000FBEC00F001EEBCF0EE5003E003EC01F0EB
:10723000FBD70D0E03EC01F00A0E03EC01F08FC139
:1072400010F001018E512DEC01F0D896B8A7D88628
:107250000001D8B64BEF39F001EEBCF0020E016E22
:10726000066A87C112F086C111F0CCEC00F0EF6A1B
:10727000150EF76E980EF66EFBEC00F001EEBCF00A
:10728000EE5003E003EC01F0FBD70D0E03EC01F030
:107290000A0E03EC01F0D8960101B8A7D8860001C8
:1072A000D8B672EF39F001EEBCF0020E016E066A3C
:1072B0007DC112F07CC111F0CCEC00F0EF6A150E2C
:1072C000F76EAA0EF66EFBEC00F001EEBCF0EE508D
:1072D00003E003EC01F0FBD70D0E03EC01F00A0E06
:1072E00003EC01F0820E026E040E076E87C104F0FB
:1072F00086C103F07DC112F07CC111F031EC00F0C9
:10730000D8960101B8A7D8860001D8B6A7EF39F002
:1073100001EEBCF0020E016E066A91C112F090C13E
:1073200011F0CCEC00F0EF6A150EF76EBC0EF66EA5
:10733000FBEC00F001EEBCF0EE5003E003EC01F0DA
:10734000FBD70D0E03EC01F00A0E03EC01F091C126
:1073500010F0010190512DEC01F0D896B8A7D88615
:107360000001D8B6D3EF39F001EEBCF0020E016E89
:10737000066A89C112F088C111F0CCEC00F0EF6A06
:10738000150EF76ECE0EF66EFBEC00F001EEBCF0C3
:10739000EE5003E003EC01F0FBD70D0E03EC01F01F
:1073A0000A0E03EC01F0D8960101B8A7D8860001B7
:1073B000D8B6FAEF39F001EEBCF0020E016E066AA3
:1073C0007FC112F07EC111F0CCEC00F0EF6A150E17
:1073D000F76EE00EF66EFBEC00F001EEBCF0EE5046
:1073E00003E003EC01F0FBD70D0E03EC01F00A0EF5
:1073F00003EC01F0820E026E040E076E89C104F0E8
:1074000088C103F07FC112F07EC111F031EC00F0B1
:10741000D8960101B8A7D8860001D8B62FEF3AF068
:1074200001EEBCF0020E016E066A93C112F092C129
:1074300011F0CCEC00F0EF6A150EF76EF20EF66E5E
:10744000FBEC00F001EEBCF0EE5003E003EC01F0C9
:10745000FBD70D0E03EC01F00A0E03EC01F093C113
:1074600010F0010192512DEC01F0D896B8A7D88602
:107470000001D8B661EF3AF001EEBCF0020E016EE9
:10748000066A95C112F094C111F0CCEC00F0EF6ADD
:107490000D0E03EC01F00A0E03EC01F0160EF76E70
:1074A000040EF66EFBEC00F001EEBCF0EE5003E0D3
:1074B00003EC01F0FBD70D0E03EC01F00A0E03EC18
:1074C00001F095C110F0010194512DEC01F0949858
:1074D000829800011200D8960101B8A7D886000151
:1074E000D8B698EF3AF001EEBCF0020E016E066AD3
:1074F00097C112F096C111F0CCEC00F0EF6A0D0EBE
:1075000003EC01F00A0E03EC01F0160EF76E160EF6
:10751000F66EFBEC00F001EEBCF0EE5003E003EC85
:1075200001F0FBD70D0E03EC01F00A0E03EC01F0A5
:1075300097C110F0010196512DEC01F0D896B8A733
:10754000D8860001D8B6C4EF3AF001EEBCF0020EC6
:10755000016E066AA3C112F0A2C111F0CCEC00F0DA
:10756000EF6A160EF76E280EF66EFBEC00F001EED9
:10757000BCF0EE5003E003EC01F0FBD70D0E03EC82
:1075800001F00A0E03EC01F0D8960101B8A7D886E5
:107590000001D8B6EBEF3AF001EEBCF0020E016E3E
:1075A000066A99C112F098C111F0CCEC00F0EF6AB4
:1075B000160EF76E3A0EF66EFBEC00F001EEBCF024
:1075C000EE5003E003EC01F0FBD70D0E03EC01F0ED
:1075D0000A0E03EC01F0820E026E020E076EA3C1CA
:1075E00004F0A2C103F099C112F098C111F031EC7E
:1075F00000F0D8960101B8A7D8860001D8B620EFD0
:107600003BF001EEBCF0020E016E066AADC112F055
:10761000ACC111F0CCEC00F0EF6A160EF76E4C0E18
:10762000F66EFBEC00F001EEBCF0EE5003E003EC74
:1076300001F0FBD70D0E03EC01F00A0E03EC01F094
:10764000ADC110F00101AC512DEC01F0D896B8A7F6
:10765000D8860001D8B64CEF3BF001EEBCF0020E2C
:10766000016E066AA5C112F0A4C111F0CCEC00F0C5
:10767000EF6A160EF76E5E0EF66EFBEC00F001EE92
:10768000BCF0EE5003E003EC01F0FBD70D0E03EC71
:1076900001F00A0E03EC01F0D8960101B8A7D886D4
:1076A0000001D8B673EF3BF001EEBCF0020E016EA4
:1076B000066A9BC112F09AC111F0CCEC00F0EF6A9F
:1076C000160EF76E700EF66EFBEC00F001EEBCF0DD
:1076D000EE5003E003EC01F0FBD70D0E03EC01F0DC
:1076E0000A0E03EC01F0820E026E020E076EA5C1B7
:1076F00004F0A4C103F09BC112F09AC111F031EC67
:1077000000F0D8960101B8A7D8860001D8B6A8EF36
:107710003BF001EEBCF0020E016E066AAFC112F042
:10772000AEC111F0CCEC00F0EF6A160EF76E820ECF
:10773000F66EFBEC00F001EEBCF0EE5003E003EC63
:1077400001F0FBD70D0E03EC01F00A0E03EC01F083
:10775000AFC110F00101AE512DEC01F0D896B8A7E1
:10776000D8860001D8B6D4EF3BF001EEBCF0020E93
:10777000016E066AA7C112F0A6C111F0CCEC00F0B0
:10778000EF6A160EF76E940EF66EFBEC00F001EE4B
:10779000BCF0EE5003E003EC01F0FBD70D0E03EC60
:1077A00001F00A0E03EC01F0D8960101B8A7D886C3
:1077B0000001D8B6FBEF3BF001EEBCF0020E016E0B
:1077C000066A9DC112F09CC111F0CCEC00F0EF6A8A
:1077D000160EF76EA60EF66EFBEC00F001EEBCF096
:1077E000EE5003E003EC01F0FBD70D0E03EC01F0CB
:1077F0000A0E03EC01F0820E026E020E076EA7C1A4
:1078000004F0A6C103F09DC112F09CC111F031EC4F
:1078100000F0D8960101B8A7D8860001D8B630EF9D
:107820003CF001EEBCF0020E016E066AB1C112F02E
:10783000B0C111F0CCEC00F0EF6A160EF76EB80E86
:10784000F66EFBEC00F001EEBCF0EE5003E003EC52
:1078500001F0FBD70D0E03EC01F00A0E03EC01F072
:10786000B1C110F00101B0512DEC01F0D896B8A7CC
:10787000D8860001D8B65CEF3CF001EEBCF0020EF9
:10788000016E066AA9C112F0A8C111F0CCEC00F09B
:10789000EF6A160EF76ECA0EF66EFBEC00F001EE04
:1078A000BCF0EE5003E003EC01F0FBD70D0E03EC4F
:1078B00001F00A0E03EC01F0D8960101B8A7D886B2
:1078C0000001D8B683EF3CF001EEBCF0020E016E71
:1078D000066A9FC112F09EC111F0CCEC00F0EF6A75
:1078E000160EF76EDC0EF66EFBEC00F001EEBCF04F
:1078F000EE5003E003EC01F0FBD70D0E03EC01F0BA
:107900000A0E03EC01F0820E026E020E076EA9C190
:1079100004F0A8C103F09FC112F09EC111F031EC38
:1079200000F0D8960101B8A7D8860001D8B6B8EF04
:107930003CF001EEBCF0020E016E066AB3C112F01B
:10794000B2C111F0CCEC00F0EF6A160EF76EEE0E3D
:10795000F66EFBEC00F001EEBCF0EE5003E003EC41
:1079600001F0FBD70D0E03EC01F00A0E03EC01F061
:10797000B3C110F00101B2512DEC01F0D896B8A7B7
:10798000D8860001D8B6E4EF3CF001EEBCF0020E60
:10799000016E066AABC112F0AAC111F0CCEC00F086
:1079A000EF6A170EF76E000EF66EFBEC00F001EEBC
:1079B000BCF0EE5003E003EC01F0FBD70D0E03EC3E
:1079C00001F00A0E03EC01F0D8960101B8A7D886A1
:1079D0000001D8B60BEF3DF001EEBCF0020E016ED7
:1079E000066AA1C112F0A0C111F0CCEC00F0EF6A60
:1079F000170EF76E120EF66EFBEC00F001EEBCF007
:107A0000EE5003E003EC01F0FBD70D0E03EC01F0A8
:107A10000A0E03EC01F0820E026E020E076EABC17D
:107A200004F0AAC103F0A1C112F0A0C111F031EC21
:107A300000F0D8960101B8A7D8860001D8B640EF6B
:107A40003DF001EEBCF0020E016E066AB5C112F007
:107A5000B4C111F0CCEC00F0EF6A170EF76E240EF3
:107A6000F66EFBEC00F001EEBCF0EE5003E003EC30
:107A700001F0FBD70D0E03EC01F00A0E03EC01F050
:107A8000B5C110F00101B4512DEC01F0D896B8A7A2
:107A9000D8860001D8B672EF3DF001EEBCF0020EC0
:107AA000016E066AB7C112F0B6C111F0CCEC00F05D
:107AB000EF6A0D0E03EC01F00A0E03EC01F0170E55
:107AC000F76E360EF66EFBEC00F001EEBCF0EE50F9
:107AD00003E003EC01F0FBD70D0E03EC01F00A0EFE
:107AE00003EC01F0B7C110F00101B6512DEC01F02B
:107AF000000112000D0E03EC01F00A0E03EC01F080
:107B00000D0E03EC01F00A0E03EC01F0170EF76EF8
:107B1000480EF66EFBEC00F00D0E03EC01F00A0EC1
:107B200003EC01F0170EF76E640EF66EFBEC00F03E
:107B30000D0E03EC01F00A0E03EC01F0170EF76EC8
:107B40009A0EF66EFBEC00F00D0E03EC01F00A0E3F
:107B500003EC01F0170EF76ED00EF66EFBEC00F0A2
:107B60000D0E03EC01F00A0E03EC01F0180EF76E97
:107B7000060EF66EFBEC00F00D0E03EC01F00A0EA3
:107B800003EC01F0180EF76E3C0EF66EFBEC00F005
:107B90000D0E03EC01F00A0E03EC01F0180EF76E67
:107BA000720EF66EFBEC00F00D0E03EC01F00A0E07
:107BB00003EC01F0180EF76EA80EF66EFBEC00F069
:107BC0000D0E03EC01F00A0E03EC01F0180EF76E37
:107BD000DE0EF66EFBEC00F00D0E03EC01F00A0E6B
:107BE00003EC01F0190EF76E140EF66EFBEC00F0CC
:107BF0000D0E03EC01F00A0E03EC01F0190EF76E06
:107C00004A0EF66EFBEC00F00D0E03EC01F00A0ECE
:107C100003EC01F0190EF76E800EF66EFBEC00F02F
:107C20000D0E03EC01F00A0E03EC01F0190EF76ED5
:107C3000B20EF66EFBEC00F00D0E03EC01F00A0E36
:107C400003EC01F00D0E03EC01F00A0E03EC01F061
:107C500012000D0E03EC01F00A0E03EC01F0190EF8
:107C6000F76EDC0EF66EFBEC00F00D0E03EC01F08F
:107C70000A0E03EC01F00D0E03EC01F00A0E03EC0A
:107C800001F0190EF76EEC0EF66EFBEC00F00D0E27
:107C900003EC01F00A0E03EC01F00D0E03EC01F011
:107CA0000A0E03EC01F01A0EF76E1A0EF66EFBECDC
:107CB00000F00D0E03EC01F00A0E03EC01F00D0EC6
:107CC00003EC01F00A0E03EC01F01A0EF76E960EAB
:107CD000F66EFBEC00F00D0E03EC01F00A0E03EC67
:107CE00001F01A0EF76ECC0EF66EFBEC00F00D0EE6
:107CF00003EC01F00A0E03EC01F01B0EF76E0C0E04
:107D0000F66EFBEC00F00D0E03EC01F00A0E03EC36
:107D100001F00D0E03EC01F00A0E03EC01F01B0E56
:107D2000F76E640EF66EFBEC00F00D0E03EC01F046
:107D30000A0E03EC01F00D0E03EC01F00A0E03EC49
:107D400001F01B0EF76EC40EF66EFBEC00F00D0E8C
:107D500003EC01F00A0E03EC01F00D0E03EC01F050
:107D60000A0E03EC01F01C0EF76E400EF66EFBECF3
:107D700000F00D0E03EC01F00A0E03EC01F01C0EF6
:107D8000F76E760EF66EFBEC00F00D0E03EC01F0D4
:107D90000A0E03EC01F01C0EF76EB60EF66EFBEC4D
:107DA00000F00D0E03EC01F00A0E03EC01F00D0ED5
:107DB00003EC01F00A0E03EC01F01D0EF76E0E0E3F
:107DC000F66EFBEC00F00D0E03EC01F00A0E03EC76
:107DD00001F00D0E03EC01F00A0E03EC01F01D0E94
:107DE000F76E6E0EF66EFBEC00F00D0E03EC01F07C
:107DF0000A0E03EC01F00D0E03EC01F00A0E03EC89
:107E000001F01D0EF76EAC0EF66EFBEC00F00D0EE1
:107E100003EC01F00A0E03EC01F01D0EF76EE20E0A
:107E2000F66EFBEC00F00D0E03EC01F00A0E03EC15
:107E300001F01E0EF76E100EF66EFBEC00F00D0E4C
:107E400003EC01F00A0E03EC01F00D0E03EC01F05F
:107E50000A0E03EC01F01E0EF76E4E0EF66EFBECF2
:107E600000F00D0E03EC01F00A0E03EC01F01E0E03
:107E7000F76E760EF66EFBEC00F00D0E03EC01F0E3
:107E80000A0E03EC01F01E0EF76EA00EF66EFBEC70
:107E900000F00D0E03EC01F00A0E03EC01F01E0ED3
:107EA000F76ECA0EF66EFBEC00F00D0E03EC01F05F
:107EB0000A0E03EC01F01E0EF76EFC0EF66EFBECE4
:107EC00000F00D0E03EC01F00A0E03EC01F01F0EA2
:107ED000F76E260EF66EFBEC00F00D0E03EC01F0D3
:107EE0000A0E03EC01F01F0EF76E520EF66EFBEC5D
:107EF00000F00D0E03EC01F00A0E03EC01F01F0E72
:107F0000F76E700EF66EFBEC00F00D0E03EC01F058
:107F10000A0E03EC01F00D0E03EC01F00A0E03EC67
:107F200001F012000D0E03EC01F00A0E03EC01F05B
:107F30001F0EF76E8E0EF66EFBEC00F00D0E03ECCE
:107F400001F00A0E03EC01F001EEBCF0020E016E2E
:107F500001016851C9EC00F0EF6A1F0EF76E960E32
:107F6000F66EFBEC00F001EEBCF0EE5003E003EC2B
:107F700001F0FBD70D0E03EC01F00A0E03EC01F04B
:107F800001EEBCF0020E016E066A6CC112F06BC10C
:107F900011F0CCEC00F0EF6A1F0EF76EA80EF66E33
:107FA000FBEC00F001EEBCF0EE5003E003EC01F05E
:107FB000FBD70D0E03EC01F00A0E03EC01F001EE0D
:107FC000BCF0020E016E066A6FC112F06EC111F0B4
:107FD000CCEC00F0EF6A1F0EF76EBC0EF66EFBECF9
:107FE00000F001EEBCF0EE5003E003EC01F0FBD733
:107FF0000D0E03EC01F00A0E03EC01F01F0EF76EFC
:10800000D00EF66EFBEC00F00D0E03EC01F00A0E44
:1080100003EC01F001EEBCF0020E016E066A75C1C0
:1080200012F074C111F0CCEC00F0EF6A1F0EF76E85
:10803000E80EF66EFBEC00F001EEBCF0EE5003E053
:1080400003EC01F0FBD70D0E03EC01F00A0E03EC7C
:1080500001F001EEBCF0020E016E066A77C112F06B
:1080600076C111F0CCEC00F0EF6A1F0EF76EFC0E3B
:10807000F66EFBEC00F001EEBCF0EE5003E003EC1A
:1080800001F0FBD70D0E03EC01F00A0E03EC01F03A
:1080900001EEBCF0020E016E066A81C112F080C1D1
:1080A00011F0CCEC00F0EF6A200EF76E160EF66EB3
:1080B000FBEC00F001EEBCF0EE5003E003EC01F04D
:1080C000FBD70D0E03EC01F00A0E03EC01F001EEFC
:1080D000BCF0020E016E066A8BC112F08AC111F06B
:1080E000CCEC00F0EF6A200EF76E300EF66EFBEC73
:1080F00000F001EEBCF0EE5003E003EC01F0FBD722
:108100000D0E03EC01F00A0E03EC01F001EEBCF0E1
:10811000020E016E066A79C112F078C111F0CCEC42
:1081200000F0EF6A200EF76E4A0EF66EFBEC00F0E0
:1081300001EEBCF0EE5003E003EC01F0FBD70D0EB6
:1081400003EC01F00A0E03EC01F001EEBCF0020EAC
:10815000016E066A83C112F082C111F0CCEC00F00E
:10816000EF6A200EF76E640EF66EFBEC00F001EE87
:10817000BCF0EE5003E003EC01F0FBD70D0E03EC76
:1081800001F00A0E03EC01F001EEBCF0020E016EEC
:10819000066A8DC112F08CC111F0CCEC00F0EF6AD0
:1081A000200EF76E7E0EF66EFBEC00F001EEBCF0DA
:1081B000EE5003E003EC01F0FBD70D0E03EC01F0F1
:1081C0000A0E03EC01F001EEBCF0020E016E066A2D
:1081D0007BC112F07AC111F0CCEC00F0EF6A200EF6
:1081E000F76E980EF66EFBEC00F001EEBCF0EE5070
:1081F00003E003EC01F0FBD70D0E03EC01F00A0ED7
:1082000003EC01F001EEBCF0020E016E066A85C1BE
:1082100012F084C111F0CCEC00F0EF6A200EF76E82
:10822000B20EF66EFBEC00F001EEBCF0EE5003E097
:1082300003EC01F0FBD70D0E03EC01F00A0E03EC8A
:1082400001F001EEBCF0020E016E066A8FC112F061
:108250008EC111F0CCEC00F0EF6A200EF76ECC0E60
:10826000F66EFBEC00F001EEBCF0EE5003E003EC28
:1082700001F0FBD70D0E03EC01F00A0E03EC01F048
:1082800001EEBCF0020E016E066A7DC112F07CC1E7
:1082900011F0CCEC00F0EF6A200EF76EE60EF66EF1
:1082A000FBEC00F001EEBCF0EE5003E003EC01F05B
:1082B000FBD70D0E03EC01F00A0E03EC01F001EE0A
:1082C000BCF0020E016E066A87C112F086C111F081
:1082D000CCEC00F0EF6A210EF76E000EF66EFBECB0
:1082E00000F001EEBCF0EE5003E003EC01F0FBD730
:1082F0000D0E03EC01F00A0E03EC01F001EEBCF0F0
:10830000020E016E066A91C112F090C111F0CCEC20
:1083100000F0EF6A210EF76E1A0EF66EFBEC00F01D
:1083200001EEBCF0EE5003E003EC01F0FBD70D0EC4
:1083300003EC01F00A0E03EC01F001EEBCF0020EBA
:10834000016E066A7FC112F07EC111F0CCEC00F024
:10835000EF6A210EF76E340EF66EFBEC00F001EEC4
:10836000BCF0EE5003E003EC01F0FBD70D0E03EC84
:1083700001F00A0E03EC01F001EEBCF0020E016EFA
:10838000066A89C112F088C111F0CCEC00F0EF6AE6
:10839000210EF76E4E0EF66EFBEC00F001EEBCF017
:1083A000EE5003E003EC01F0FBD70D0E03EC01F0FF
:1083B0000A0E03EC01F001EEBCF0020E016E066A3B
:1083C00093C112F092C111F0CCEC00F0EF6A210ED3
:1083D000F76E680EF66EFBEC00F001EEBCF0EE50AE
:1083E00003E003EC01F0FBD70D0E03EC01F00A0EE5
:1083F00003EC01F001EEBCF0020E016E066A95C1BD
:1084000012F094C111F0CCEC00F0EF6A210EF76E7F
:10841000820EF66EFBEC00F001EEBCF0EE5003E0D5
:1084200003EC01F0FBD70D0E03EC01F00A0E03EC98
:1084300001F0210EF76E9C0EF66EFBEC00F00D0EB7
:1084400003EC01F00A0E03EC01F001EEBCF0020EA9
:10845000016E066A97C112F096C111F0CCEC00F0E3
:10846000EF6A210EF76EB40EF66EFBEC00F001EE33
:10847000BCF0EE5003E003EC01F0FBD70D0E03EC73
:1084800001F00A0E03EC01F001EEBCF0020E016EE9
:10849000066A99C112F098C111F0CCEC00F0EF6AB5
:1084A000210EF76ECE0EF66EFBEC00F001EEBCF086
:1084B000EE5003E003EC01F0FBD70D0E03EC01F0EE
:1084C0000A0E03EC01F001EEBCF0020E016E066A2A
:1084D000A3C112F0A2C111F0CCEC00F0EF6A210EA2
:1084E000F76EE80EF66EFBEC00F001EEBCF0EE501D
:1084F00003E003EC01F0FBD70D0E03EC01F00A0ED4
:1085000003EC01F001EEBCF0020E016E066AADC193
:1085100012F0ACC111F0CCEC00F0EF6A220EF76E55
:10852000020EF66EFBEC00F001EEBCF0EE5003E044
:1085300003EC01F0FBD70D0E03EC01F00A0E03EC87
:1085400001F001EEBCF0020E016E066A9BC112F052
:108550009AC111F0CCEC00F0EF6A220EF76E1C0EFF
:10856000F66EFBEC00F001EEBCF0EE5003E003EC25
:1085700001F0FBD70D0E03EC01F00A0E03EC01F045
:1085800001EEBCF0020E016E066AA5C112F0A4C194
:1085900011F0CCEC00F0EF6A220EF76E360EF66E9C
:1085A000FBEC00F001EEBCF0EE5003E003EC01F058
:1085B000FBD70D0E03EC01F00A0E03EC01F001EE07
:1085C000BCF0020E016E066AAFC112F0AEC111F02E
:1085D000CCEC00F0EF6A220EF76E500EF66EFBEC5C
:1085E00000F001EEBCF0EE5003E003EC01F0FBD72D
:1085F0000D0E03EC01F00A0E03EC01F001EEBCF0ED
:10860000020E016E066A9DC112F09CC111F0CCEC05
:1086100000F0EF6A220EF76E6A0EF66EFBEC00F0C9
:1086200001EEBCF0EE5003E003EC01F0FBD70D0EC1
:1086300003EC01F00A0E03EC01F001EEBCF0020EB7
:10864000016E066AA7C112F0A6C111F0CCEC00F0D1
:10865000EF6A220EF76E840EF66EFBEC00F001EE70
:10866000BCF0EE5003E003EC01F0FBD70D0E03EC81
:1086700001F00A0E03EC01F001EEBCF0020E016EF7
:10868000066AB1C112F0B0C111F0CCEC00F0EF6A93
:10869000220EF76E9E0EF66EFBEC00F001EEBCF0C3
:1086A000EE5003E003EC01F0FBD70D0E03EC01F0FC
:1086B0000A0E03EC01F001EEBCF0020E016E066A38
:1086C0009FC112F09EC111F0CCEC00F0EF6A220EB7
:1086D000F76EB80EF66EFBEC00F001EEBCF0EE505B
:1086E00003E003EC01F0FBD70D0E03EC01F00A0EE2
:1086F00003EC01F001EEBCF0020E016E066AA9C1A6
:1087000012F0A8C111F0CCEC00F0EF6A220EF76E67
:10871000D20EF66EFBEC00F001EEBCF0EE5003E082
:1087200003EC01F0FBD70D0E03EC01F00A0E03EC95
:1087300001F001EEBCF0020E016E066AB3C112F048
:10874000B2C111F0CCEC00F0EF6A220EF76EEC0E25
:10875000F66EFBEC00F001EEBCF0EE5003E003EC33
:1087600001F0FBD70D0E03EC01F00A0E03EC01F053
:1087700001EEBCF0020E016E066AA1C112F0A0C1AA
:1087800011F0CCEC00F0EF6A230EF76E060EF66ED9
:10879000FBEC00F001EEBCF0EE5003E003EC01F066
:1087A000FBD70D0E03EC01F00A0E03EC01F001EE15
:1087B000BCF0020E016E066AABC112F0AAC111F044
:1087C000CCEC00F0EF6A230EF76E200EF66EFBEC99
:1087D00000F001EEBCF0EE5003E003EC01F0FBD73B
:1087E0000D0E03EC01F00A0E03EC01F001EEBCF0FB
:1087F000020E016E066AB5C112F0B4C111F0CCECE4
:1088000000F0EF6A230EF76E3A0EF66EFBEC00F006
:1088100001EEBCF0EE5003E003EC01F0FBD70D0ECF
:1088200003EC01F00A0E03EC01F001EEBCF0020EC5
:10883000016E066AB7C112F0B6C111F0CCEC00F0BF
:10884000EF6A230EF76E540EF66EFBEC00F001EEAD
:10885000BCF0EE5003E003EC01F0FBD70D0E03EC8F
:1088600001F00A0E03EC01F00D0E03EC01F00A0E0C
:1088700003EC01F0230EF76E6E0EF66EFBEC00F0CB
:108880000D0E03EC01F00A0E03EC01F000011200E2
:1088900029EC3EF0230EF76E880EF66EFBEC00F02E
:1088A0000D0E03EC01F00A0E03EC01F012000D0EA8
:1088B00003EC01F00A0E03EC01F0230EF76EB40E88
:1088C000F66EFBEC00F00D0E03EC01F00A0E03EC6B
:1088D00001F00101686B6C6B010E6B6F6F6B010E29
:1088E0006E6F756B010E746F776B010E766F816B17
:1088F000010E806F8B6B010E8A6F796B010E786FA2
:10890000836B010E826F8D6B010E8C6F7B6B010E82
:108910007A6F856B010E846F8F6B010E8E6F7D6B8E
:10892000010E7C6F876B010E866F916B010E906F4D
:108930007F6B010E7E6F896B010E886F936B010E4A
:10894000926F956B010E946F976B010E966F996BFA
:10895000010E986FA36B010EA26FAD6B010EAC6F91
:108960009B6B010E9A6FA56B010EA46FAF6B010E8E
:10897000AE6F9D6B010E9C6FA76B010EA66FB16B66
:10898000010EB06F9F6B010E9E6FA96B010EA86F59
:10899000B36B010EB26FA16B010EA06FAB6B010E3A
:1089A000AA6FB56B010EB46FB76B010EB66F0D0EEB
:1089B00003EC01F00A0E03EC01F0000112001200BA
:020000040030CA
:03000100821A0E52
:020005008181F7
:060008000FC00FE00F40E5
:00000001FF
